:020000040800F2
:1000000000500020995A0008455100084D51000841
:10001000555100085D5100086551000800000000BE
:100020000000000000000000000000006D5100080A
:100030007951000800000000855100089151000826
:10004000E15A0008E15A0008E15A0008E15A0008A4
:10005000E15A0008E15A0008E15A0008E15A000894
:10006000E15A0008E15A0008E15A0008E15A000884
:10007000E15A00089D510008E15A0008E15A0008C1
:10008000B1510008E15A0008E15A0008E15A00089D
:10009000E15A0008E15A0008E15A0008E15A000854
:1000A000E15A0008E15A0008E15A0008E15A000844
:1000B000E15A0008C5510008E15A0008E15A000859
:1000C000E15A0008E15A0008E15A0008E15A000824
:1000D000E15A0008E15A0008D95100088953000884
:1000E000255400083D540008E15A000800000000B3
:1000F0000000000000000000000000000000000000
:0C01000000000000000000005FF808F1A3
:10010C0010B5054C237833B9044B13B10448AFF345
:10011C0000800123237010BD780000200000000037
:10012C00A470000808B5034B1BB103490348AFF397
:10013C00008008BD000000007C000020A4700008B6
:10014C00034613F8012B002AFBD1181A013870470B
:10015C0080B400AF00BFBD4680BC704780B582B094
:10016C0000AF78607B68002B01D1012341E07B68F4
:10017C0093F83D30DBB2002B06D17B68002283F86C
:10018C003C20786800F039F87B68022283F83D2027
:10019C007B681A687B6804331946104600F09CF99A
:1001AC007B68012283F846207B68012283F83E207D
:1001BC007B68012283F83F207B68012283F8402072
:1001CC007B68012283F841207B68012283F842205E
:1001DC007B68012283F843207B68012283F844204A
:1001EC007B68012283F845207B68012283F83D203F
:1001FC00002318460837BD4680BD80B483B000AFDD
:10020C00786000BF0C37BD4680BC704780B485B0A9
:10021C0000AF78607B6893F83D30DBB2012B01D0E6
:10022C0001233AE07B68022283F83D207B681B683F
:10023C00DA687B681B6842F00102DA607B681B6835
:10024C00184A93420ED07B681B68B3F1804F09D0DB
:10025C007B681B68144A934204D07B681B68134A62
:10026C00934211D17B681B689B6803F00703FB600A
:10027C00FB68062B10D07B681B681A687B681B68B0
:10028C0042F001021A6007E07B681B681A687B6801
:10029C001B6842F001021A60002318461437BD4651
:1002AC0080BC7047002C0140000400400008004056
:1002BC0080B584B000AF78607B681B68DB68FB603E
:1002CC007B681B681B69BB60BB6803F00203002BD7
:1002DC0020D0FB6803F00203002B1BD07B681B684B
:1002EC006FF002021A617B6801221A777B681B6827
:1002FC009B6903F00303002B03D0786800F0D1F85E
:10030C0005E0786800F0C4F8786800F0D3F87B68F2
:10031C0000221A77BB6803F00403002B20D0FB6883
:10032C0003F00403002B1BD07B681B686FF00402E6
:10033C001A617B6802221A777B681B689B6903F43D
:10034C004073002B03D0786800F0ABF805E07868B8
:10035C0000F09EF8786800F0ADF87B6800221A7700
:10036C00BB6803F00803002B20D0FB6803F00803E4
:10037C00002B1BD07B681B686FF008021A617B682E
:10038C0004221A777B681B68DB6903F00303002BDC
:10039C0003D0786800F085F805E0786800F078F80C
:1003AC00786800F087F87B6800221A77BB6803F046
:1003BC001003002B20D0FB6803F01003002B1BD084
:1003CC007B681B686FF010021A617B6808221A7731
:1003DC007B681B68DB6903F44073002B03D07868DF
:1003EC0000F05FF805E0786800F052F8786800F0EB
:1003FC0061F87B6800221A77BB6803F00103002BBD
:10040C000CD0FB6803F00103002B07D07B681B6842
:10041C006FF001021A61786804F076FEBB6803F095
:10042C008003002B0CD0FB6803F08003002B07D05B
:10043C007B681B686FF080021A61786800F0C3F863
:10044C00BB6803F04003002B0CD0FB6803F04003A7
:10045C00002B07D07B681B686FF040021A6178682C
:10046C0000F031F8BB6803F02003002B0CD0FB68C4
:10047C0003F02003002B07D07B681B686FF0200271
:10048C001A61786800F096F800BF1037BD4680BD41
:10049C0080B483B000AF786000BF0C37BD4680BC21
:1004AC00704780B483B000AF786000BF0C37BD4696
:1004BC0080BC704780B483B000AF786000BF0C374D
:1004CC00BD4680BC704780B483B000AF786000BF7D
:1004DC000C37BD4680BC704780B485B000AF7860E7
:1004EC0039607B681B68FB607B682F4A93420BD09A
:1004FC007B68B3F1804F07D07B682C4A934203D0C2
:10050C007B682B4A934208D1FB6823F07003FB6095
:10051C003B685B68FA681343FB607B68224A934232
:10052C000BD07B68B3F1804F07D07B681F4A934296
:10053C0003D07B681E4A934208D1FB6823F44073B6
:10054C00FB603B68DB68FA681343FB60FB6823F0D5
:10055C0080023B685B691343FB607B68FA681A6036
:10056C003B689A687B68DA623B681A687B689A62B7
:10057C007B680D4A934203D13B681A697B681A6306
:10058C007B6801225A617B681B6903F00103002B15
:10059C0005D07B681B6923F001027B681A6100BFE0
:1005AC001437BD4680BC7047002C0140000400404D
:1005BC000008004080B483B000AF786000BF0C37F7
:1005CC00BD4680BC704780B483B000AF786000BF7C
:1005DC000C37BD4680BC704780B584B000AF7860E6
:1005EC000023FB607B68002B01D101237AE07B6840
:1005FC005B7CDBB2002B05D17B6800221A74786817
:10060C0004F0B2FF7B6802225A74786800F0D5FBC4
:10061C000346002B04D07B6804225A74012361E04A
:10062C00786800F08EFC0346002B04D07B68042213
:10063C005A74012356E07B681B685A687B681B68F8
:10064C0022F007025A607B689B68002B05D0274B71
:10065C001B6B264A23F001031363244BDB6A23F440
:10066C0060727B689B6821491343CB627B685B6833
:10067C00B3F1FF3F03D07B685B68FB600EE00120A9
:10068C0001F088FBF860FB68002B04D17B68042226
:10069C005A74012326E0FB68013BFB60FB681A0CD3
:1006AC007B681B6802F00F029A607B681B68FA6813
:1006BC0092B2DA60786800F06CFC0346002B04D030
:1006CC007B6804225A7401230CE07B680022DA73E5
:1006DC007B6801225A737B6801229A737B68012222
:1006EC005A74002318461037BD4680BD006C00407C
:1006FC0090B587B000AFF860B9607A6000237B6179
:10070C0000233B61FB68002B02D0BB68002B01D19E
:10071C00012380E0FB681B7C012B01D102237AE0D2
:10072C00FB6801221A74FB6802225A747B68002B46
:10073C0013D1BB681B781A464FF4616303FB02F2BA
:10074C00BB685B7819460B461B015B1A9B00134474
:10075C00BA68927813447B611EE0BB681B7818461C
:10076C0000F05CFC03461A464FF4616303FB02F491
:10077C00BB685B78184600F051FC03461A461346DA
:10078C001B019B1A9B001C44BB689B78184600F00D
:10079C0045FC034623447B617969F86800F06AFBE9
:1007AC000346002B07D0FB6804225A74FB68002216
:1007BC001A7401232FE0FB681B685A68FB681B68DE
:1007CC0022F005025A60F86800F07BFB38613B6947
:1007DC00B3F1FF3F18D03A697B699A4214D23B6956
:1007EC0003F5A83303F5C0733B613969F86800F071
:1007FC0081FB0346002B07D0FB6804225A74FB686C
:10080C0000221A74012306E0FB6801225A74FB686B
:10081C0000221A74002318461C37BD4690BD0000F8
:10082C0080B588B000AFF860B9607A600023BB6116
:10083C000023FB6100237B6100233B61FB68002BE1
:10084C0002D0BB68002B01D10123B5E0FB681B680B
:10085C005B6803F00403002B01D00123ACE0F868C3
:10086C0000F0D8FAB861BB69554AA2FB0323DB0A36
:10087C003B61BA69524BA3FB0213DB0A4FF4616173
:10088C0001FB03F3D31A4F4AA2FB03235B09DAB231
:10089C00BB685A70BB694A4AA2FB0312D20A4FF4D6
:1008AC00616101FB02F29A1A464BA3FB0213590930
:1008BC000B461B015B1A9B00D11ACAB2BB689A701B
:1008CC003B69172B55D93B693F4AA2FB03231B09F4
:1008DC007B6139693C4BA3FB01231A0913465B006E
:1008EC001344DB00CA1AD2B2BB681A70F86800F065
:1008FC00E8FAF861FB69B3F1FF3F08D0FA69BB690C
:10090C009A4204D9FA69BB69D31AFB6102E04FF031
:10091C00FF33FB617B692D4A02FB03F3BA69D31ADF
:10092C00BB61B969F86800F0A5FA0346002B01D049
:10093C00012341E0FB69B3F1FF3F0CD0FA69BB69BD
:10094C001344FB61F969F86800F0D4FA0346002BF4
:10095C000AD0012330E0F969F86800F0CBFA0346BD
:10096C00002B01D0012327E07969F86800F073FBB4
:10097C0003E03B69DAB2BB681A707B68002B1AD0B3
:10098C00BB681B78184600F02CFB03461A46BB6864
:10099C001A70BB685B78184600F023FB03461A46B6
:1009AC00BB685A70BB689B78184600F01AFB03466C
:1009BC001A46BB689A70002318462037BD4680BD86
:1009CC00C5B3A29189888888ABAAAAAA80510100D4
:1009DC0080B588B000AFF860B9607A600023FB6125
:1009EC000023BB6100237B61FB68002B02D0BB683A
:1009FC00002B01D1012397E0FB681B7C012B01D15B
:100A0C00022391E0FB6801221A74FB6802225A74DB
:100A1C007B68002B0CD1BB68DA78FB68DA73BB6897
:100A2C005A78FB685A73BB689A78FB689A731AE019
:100A3C00BB68DB78184600F0F1FA03461A46FB68EF
:100A4C00DA73BB685B78184600F0E8FA03461A467E
:100A5C00FB685A73BB689B78184600F0DFFA0346B4
:100A6C001A46FB689A73FB68DB7B1846FB68597B5C
:100A7C00FB689B7B1A4600F0C9FB03461A46FB68D1
:100A8C001A73FB681A7BBB681A70F86800F0C2F91D
:100A9C00F861FB69264AA2FB0323DB0A7B617B69B5
:100AAC00182B3AD97B69234AA2FB03231B09224A40
:100ABC0002FB03F3FA69D31AFB61F969F86800F0D9
:100ACC00D9F90346002B07D0FB6804225A74FB6843
:100ADC0000221A74012327E0F86800F0F2F9B861DB
:100AEC00BB69B3F1FF3F18D0BA69FB699A4214D2C3
:100AFC00BB6903F5A83303F5C073BB61B969F8682A
:100B0C0000F0F8F90346002B07D0FB6804225A7456
:100B1C00FB6800221A74012306E0FB6801225A7458
:100B2C00FB6800221A74002318462037BD4680BD8E
:100B3C00C5B3A291ABAAAAAA8051010080B586B018
:100B4C0000AFF860B9607A6007F1140300210A461F
:100B5C001A800A469A70FB68002B02D0BB68002BE7
:100B6C0001D101233AE007F1140300221946F86879
:100B7C00FFF756FE0346002B01D001232EE0FB6845
:100B8C001A7BBB681A70FB68DA7BBB68DA70FB688F
:100B9C005A7BBB685A70FB689A7BBB689A707B68FF
:100BAC00002B1AD0BB68DB78184600F01AFA034603
:100BBC001A46BB68DA70BB685B78184600F011FA0D
:100BCC0003461A46BB685A70BB689B78184600F0FF
:100BDC0008FA03461A46BB689A7000231846183761
:100BEC00BD4680BD90B589B000AFF860B9607A6041
:100BFC000023FB6107F1140300210A461A800A4600
:100C0C009A70FB68002B02D0BB68002B01D101232A
:100C1C0099E0FB681B7C012B01D1022393E0FB685C
:100C2C0001221A74FB6802225A7407F11403002281
:100C3C001946F868FFF7F4FD0346002B01D0012399
:100C4C0081E03B7D1A464FF4616303FB02F27B7D2E
:100C5C0019460B461B015B1A9B001344BA7D1344C7
:100C6C00BB617B68002B13D1BB681B781A464FF411
:100C7C00616303FB02F2BB685B7819460B461B01F0
:100C8C005B1A9B001344BA6892781344FB611EE014
:100C9C00BB681B78184600F0C1F903461A464FF49E
:100CAC00616303FB02F4BB685B78184600F0B6F98D
:100CBC0003461A4613461B019B1A9B001C44BB6837
:100CCC009B78184600F0AAF903462344FB61FA69A5
:100CDC00BB699A4205D2FB6903F5A83303F5C073CF
:100CEC00FB61F969F86800F005F90346002B07D0A1
:100CFC00FB6804225A74FB6800221A74012322E058
:100D0C00FB681B685A68FB681B6822F002025A6079
:100D1C00FB681B681A68FB681B6842F002021A60C9
:100D2C000B4B1B680A4A43F400331360084B9B6857
:100D3C00074A43F400339360FB6801225A74FB6842
:100D4C0000221A74002318462437BD4690BD00BFFC
:100D5C000004014080B582B000AF78607B681B68EE
:100D6C001B6803F00203002B11D07B681B685B68C7
:100D7C0003F00203002B0AD0786800F015F87B68AA
:100D8C001B685A687B681B6822F002025A60054B8C
:100D9C004FF400325A617B6801225A7400BF083745
:100DAC00BD4680BD0004014080B483B000AF7860C4
:100DBC0000BF0C37BD4680BC704780B584B000AF17
:100DCC0078600023FB607B68002B01D101231DE0C0
:100DDC007B681B685A687B681B6822F008025A60A3
:100DEC0000F0B4FAF86009E000F0B0FA0246FB68D3
:100DFC00D31AB3F57A7F01D9032307E07B681B680C
:100E0C005B6803F00803002BEED000231846103764
:100E1C00BD4680BD80B487B000AF786000237B8274
:100E2C0000233B820023FB8100237B617B681B68D2
:100E3C009B697B827B681B68DB69FB817B681B6819
:100E4C009B693B827A8A3B8A9A4208D03B8A1A0475
:100E5C007B681B68DB699BB213437B6104E07B8A74
:100E6C001A04FB8913437B617B6918461C37BD460A
:100E7C0080BC704780B584B000AF786039600023C7
:100E8C00FB73786800F05DF80346002B02D0012359
:100E9C00FB7311E07B681B683A68120C9A617B68E3
:100EAC001B683A6892B2DA61786800F072F803460F
:100EBC00002B01D00123FB73FB7B18461037BD467A
:100ECC0080BD80B485B000AF78600023FB81002327
:100EDC00BB817B681B681B6AFB817B681B685B6A38
:100EEC00BB81FB891A04BB89134318461437BD46D2
:100EFC0080BC704780B584B000AF78603960002347
:100F0C00FB73786800F01DF80346002B02D0012318
:100F1C00FB7311E07B681B683A68120C1A627B68E1
:100F2C001B683A6892B25A62786800F032F803464D
:100F3C00002B01D00123FB73FB7B18461037BD46F9
:100F4C0080BD80B584B000AF78600023FB6000F0FA
:100F5C00FDF9F86009E000F0F9F90246FB68D31AD4
:100F6C00B3F57A7F01D903230FE07B681B685B68BC
:100F7C0003F02003002BEED07B681B685A687B685B
:100F8C001B6842F010025A60002318461037BD4609
:100F9C0080BD80B584B000AF78600023FB607B68B7
:100FAC001B685A687B681B6822F010025A6000F0BC
:100FBC00CDF9F86009E000F0C9F90246FB68D31AD4
:100FCC00B3F57A7F01D9032307E07B681B685B6864
:100FDC0003F02003002BEED0002318461037BD463B
:100FEC0080BD80B485B000AF0346FB710023FB606D
:100FFC0005E0FB680133FB60FB790A3BFB71FB7975
:10100C00092BF6D8FB68DBB21B01DAB2FB79134370
:10101C00DBB218461437BD4680BC704780B485B02F
:10102C0000AF0346FB710023FB60FB791B09DBB2AD
:10103C001A4613469B0013445B00FB60FB7903F0DC
:10104C000F03DAB2FB68DBB21344DBB21846143779
:10105C00BD4680BC704780B586B000AF7860396003
:10106C0000237B6100233B610023FB600023BB60FA
:10107C007B68DB7B7B617B685B7B3B617B689B7B01
:10108C00FB600023BB606FE03B69012B11D03B6917
:10109C00032B0ED03B69052B0BD03B69072B08D0DB
:1010AC003B69082B05D03B690A2B02D03B690C2B02
:1010BC0017D1FB681E2B03D8FB680133FB6050E093
:1010CC003B690C2B05D03B6901333B610123FB6071
:1010DC0047E001233B610123FB607B6901337B61AA
:1010EC003FE03B69042B08D03B69062B05D03B69DC
:1010FC00092B02D03B690B2B0CD1FB681D2B03D8A1
:10110C00FB680133FB602CE03B6901333B6101233D
:10111C00FB6026E03B69022B23D1FB681B2B03D819
:10112C00FB680133FB601CE0FB681C2B11D17B6955
:10113C009BB2184600F038F80346002B03D0FB682E
:10114C000133FB600DE03B6901333B610123FB6024
:10115C0007E0FB681D2B04D13B6901333B61012384
:10116C00FB60BB680133BB60BA683B689A428BD3A7
:10117C007B69DAB27B68DA733B69DAB27B685A73E3
:10118C00FB68DAB27B689A733B69DBB2FA68D2B25D
:10119C001946786900F03AF803461A467B681A73C8
:1011AC0000BF1837BD4680BD80B483B000AF034686
:1011BC00FB80FB8803F003039BB2002B01D00023C0
:1011CC001DE0FB88104AA2FB03125209642101FBAB
:1011DC0002F29B1A9BB2002B01D001230FE0FB887B
:1011EC00094AA2FB0312D2094FF4C87101FB02F2A7
:1011FC009B1A9BB2002B01D1012300E0002318465F
:10120C000C37BD4680BC70471F85EB5180B485B050
:10121C0000AF78600B46FB701346BB700023BB60BD
:10122C000023FB607B6803F5FA63BB60FB78022B41
:10123C002DD8FA7813465B001344DB009B1A2C4A1A
:10124C00A2FB03235A08BB781A44BB681A44BB6838
:10125C00013B9B081A44BB68013B2649A1FB0313C5
:10126C005B09D21ABB68013B2249A1FB0313DB09C2
:10127C0013441A1D204BA3FB0213D11A49080B442B
:10128C0099080B46DB005B1AD31AFB6029E0FA784D
:10129C0013465B001344DB009B1A154AA2FB032385
:1012AC005A08BB781A44BB681A44BB689B081A449A
:1012BC00BB681049A1FB03135B09D21ABB680D492B
:1012CC00A1FB0313DB0913449A1C0B4BA3FB021366
:1012DC00D11A49080B4499080B46DB005B1AD31A48
:1012EC00FB60FB68DBB218461437BD4680BC704708
:1012FC00398EE3381F85EB512549922480B500AF18
:10130C00084B1B68074A43F010031360032001F0DD
:10131C000FFB0F2004F07AFA04F0F4F800231846BF
:10132C0080BD00BF0020024080B400AF054B1B788D
:10133C001A46054B1B681344034A136000BFBD4695
:10134C0080BC7047080000209400002080B400AFDF
:10135C00024B1B681846BD4680BC704794000020A9
:10136C0080B584B000AF7860FFF7F0FFB8607B68A1
:10137C00FB60FB68B3F1FF3F05D00A4B1B781A46A4
:10138C00FB681344FB6000BFFFF7E0FF0246BB683D
:10139C00D31AFA689A42F7D800BF00BF1037BD467F
:1013AC0080BD00BF0800002080B586B000AF78601B
:1013BC007B68002B01D1012372E27B681B6803F070
:1013CC000103002B00F08780924B5B6803F00C0349
:1013DC00042B0CD08F4B5B6803F00C03082B12D141
:1013EC008C4B5B6803F48033B3F5803F0BD1894B96
:1013FC001B6803F40033002B6CD07B685B68002BFC
:10140C0068D101234CE27B685B68B3F5803F06D161
:10141C00804B1B687F4A43F4803313602EE07B685B
:10142C005B68002B0CD17B4B1B687A4A23F480330E
:10143C001360784B1B68774A23F4802313601DE0FC
:10144C007B685B68B3F5A02F0CD1724B1B68714A9B
:10145C0043F4802313606F4B1B686E4A43F4803354
:10146C0013600BE06B4B1B686A4A23F480331360E8
:10147C00684B1B68674A23F4802313607B685B68A6
:10148C00002B13D0FFF762FF386108E0FFF75EFF17
:10149C0002463B69D31A642B01D9032300E25D4B4E
:1014AC001B6803F40033002BF0D014E0FFF74EFF61
:1014BC00386108E0FFF74AFF02463B69D31A642BF8
:1014CC0001D90323ECE1534B1B6803F40033002BCD
:1014DC00F0D100E000BF7B681B6803F00203002B17
:1014EC0063D04C4B5B6803F00C03002B0BD0494BC7
:1014FC005B6803F00C03082B1CD1464B5B6803F4B0
:10150C008033002B16D1434B1B6803F00203002BD6
:10151C0005D07B681B69012B01D00123C0E13D4B39
:10152C001B6823F0F8027B685B69DB0039491343C5
:10153C000B603AE07B681B69002B20D0364B0122F4
:10154C001A60FFF703FF386108E0FFF7FFFE024661
:10155C003B69D31A022B01D90323A1E12D4B1B6844
:10156C0003F00203002BF0D02A4B1B6823F0F80287
:10157C007B685B69DB00274913430B6015E0264B46
:10158C0000221A60FFF7E2FE386108E0FFF7DEFE8A
:10159C0002463B69D31A022B01D9032380E11D4B70
:1015AC001B6803F00203002BF0D17B681B6803F06F
:1015BC000803002B3AD07B689B69002B19D0174B82
:1015CC0001221A60FFF7C2FE386108E0FFF7BEFE89
:1015DC0002463B69D31A022B01D9032360E10D4B60
:1015EC005B6A03F00203002BF0D0012000F0FEFA3E
:1015FC001CE00A4B00221A60FFF7A8FE38610FE0CE
:10160C00FFF7A4FE02463B69D31A022B08D9032329
:10161C0046E100BF001002400000424280044242FA
:10162C00924B5B6A03F00203002BE9D17B681B68C9
:10163C0003F00403002B00F0A6800023FB758B4BFA
:10164C00DB6903F08053002B0DD1884BDB69874A93
:10165C0043F08053D361854BDB6903F08053BB604F
:10166C00BB680123FB75824B1B6803F48073002B52
:10167C0018D17F4B1B687E4A43F480731360FFF7CD
:10168C0065FE386108E0FFF761FE02463B69D31A3C
:10169C00642B01D9032303E1754B1B6803F480739E
:1016AC00002BF0D07B68DB68012B06D16F4B1B6ADB
:1016BC006E4A43F0010313622DE07B68DB68002B5C
:1016CC000CD16A4B1B6A694A23F001031362674B06
:1016DC001B6A664A23F0040313621CE07B68DB6818
:1016EC00052B0CD1614B1B6A604A43F00403136257
:1016FC005E4B1B6A5D4A43F0010313620BE05B4BCC
:10170C001B6A5A4A23F001031362584B1B6A574A4F
:10171C0023F0040313627B68DB68002B15D0FFF702
:10172C0015FE38610AE0FFF711FE02463B69D31A39
:10173C0041F28832934201D90323B1E04B4B1B6A2F
:10174C0003F00203002BEED014E0FFF7FFFD38612D
:10175C000AE0FFF7FBFD02463B69D31A41F28832DF
:10176C00934201D903239BE0404B1B6A03F0020315
:10177C00002BEED1FB7D012B05D13C4BDB693B4AA9
:10178C0023F08053D3617B68DB69002B00F08780EA
:10179C00364B5B6803F00C03082B61D07B68DB696C
:1017AC00022B46D1334B00221A60FFF7CFFD386174
:1017BC0008E0FFF7CBFD02463B69D31A022B01D997
:1017CC0003236DE0294B1B6803F00073002BF0D151
:1017DC007B681B6AB3F5803F08D1244B5B6823F40C
:1017EC0000327B689B68214913434B601F4B5B683D
:1017FC0023F474127B68196A7B685B6A0B431B4980
:10180C0013434B601B4B01221A60FFF79FFD38619D
:10181C0008E0FFF79BFD02463B69D31A022B01D966
:10182C0003233DE0114B1B6803F00073002BF0D039
:10183C0035E0104B00221A60FFF788FD386108E094
:10184C00FFF784FD02463B69D31A022B01D903230F
:10185C0026E0064B1B6803F00073002BF0D11EE052
:10186C007B68DB69012B07D1012319E000100240D2
:10187C0000700040600042420B4B5B68FB60FB68F1
:10188C0003F480327B681B6A9A4206D1FB6803F42E
:10189C0070127B685B6A9A4201D0012300E000233E
:1018AC0018461837BD4680BD0010024080B584B084
:1018BC0000AF786039607B68002B01D10123D0E048
:1018CC006A4B1B6803F007033A689A4210D9674BBE
:1018DC001B6823F0070265493B6813430B60634B9D
:1018EC001B6803F007033A689A4201D00123B8E061
:1018FC007B681B6803F00203002B20D07B681B68FD
:10190C0003F00403002B05D0594B5B68584A43F491
:10191C00E06353607B681B6803F00803002B05D061
:10192C00534B5B68524A43F460535360504B5B68B3
:10193C0023F0F0027B689B684D4913434B607B6836
:10194C001B6803F00103002B40D07B685B68012B04
:10195C0007D1474B1B6803F40033002B15D101232F
:10196C007FE07B685B68022B07D1414B1B6803F05F
:10197C000073002B09D1012373E03D4B1B6803F06E
:10198C000203002B01D101236BE0394B5B6823F080
:10199C0003027B685B68364913434B60FFF7D6FC48
:1019AC00F8600AE0FFF7D2FC0246FB68D31A41F25A
:1019BC008832934201D9032353E02D4B5B6803F02B
:1019CC000C027B685B689B009A42EBD1274B1B682F
:1019DC0003F007033A689A4210D2244B1B6823F099
:1019EC00070222493B6813430B60204B1B6803F032
:1019FC0007033A689A4201D0012332E07B681B68E6
:101A0C0003F00403002B08D0194B5B6823F4E0624D
:101A1C007B68DB68164913434B607B681B6803F0DB
:101A2C000803002B09D0124B5B6823F460527B68CF
:101A3C001B69DB000E4913434B6000F021F8024692
:101A4C000B4B5B681B0903F00F030A49CB5C22FAB2
:101A5C0003F3094A1360094B1B68184603F0D6FEC2
:101A6C00002318461037BD4680BD00BF0020024041
:101A7C0000100240B8740008000000200400002090
:101A8C0080B487B000AF0023FB600023BB60002351
:101A9C007B6100237B6000233B611E4B5B68FB601A
:101AAC00FB6803F00C03042B02D0082B03D027E0B7
:101ABC00194B3B6127E0FB689B0C03F00F03174AA3
:101ACC00D35C7B60FB6803F48033002B10D0114B8C
:101ADC005B685B0C03F00103114AD35CBB607B6851
:101AEC000D4A03FB02F2BB68B2FBF3F37B6104E02B
:101AFC007B680C4A02FB03F37B617B693B6102E070
:101B0C00054B3B6100BF3B6918461C37BD4680BC8A
:101B1C00704700BF0010024000127A00D074000819
:101B2C00E074000800093D0080B400AF024B1B6854
:101B3C001846BD4680BC70470000002080B500AF41
:101B4C00FFF7F2FF0246054B5B681B0A03F0070325
:101B5C000349CB5C22FA03F3184680BD0010024007
:101B6C00C874000880B500AFFFF7DEFF0246054BD6
:101B7C005B68DB0A03F007030349CB5C22FA03F32F
:101B8C00184680BD00100240C874000880B483B0B1
:101B9C0000AF786039607B680F221A60114B5B686C
:101BAC0003F003027B685A600E4B5B6803F0F00293
:101BBC007B689A600B4B5B6803F4E0627B68DA60CD
:101BCC00084B5B68DB0803F4E0627B681A61064B28
:101BDC001B6803F007023B681A6000BF0C37BD4658
:101BEC0080BC7047001002400020024080B485B0D9
:101BFC0000AF78600A4B1B680A4AA2FB03235B0AFE
:101C0C007A6802FB03F3FB6000BFFB685A1EFA60A4
:101C1C00002BF9D100BF00BF1437BD4680BC704704
:101C2C0000000020D34D621080B586B000AF786004
:101C3C0000233B610023FB607B681B6803F00103FE
:101C4C00002B7DD00023FB754F4BDB6903F08053D9
:101C5C00002B0DD14C4BDB694B4A43F08053D361C5
:101C6C00494BDB6903F08053BB60BB680123FB75F8
:101C7C00464B1B6803F48073002B18D1434B1B6835
:101C8C00424A43F480731360FFF760FB386108E04D
:101C9C00FFF75CFB02463B69D31A642B01D9032383
:101CAC006DE03A4B1B6803F48073002BF0D0364B7D
:101CBC001B6A03F44073FB60FB68002B2ED07B681F
:101CCC005B6803F44073FA689A4227D02E4B1B6A68
:101CDC0023F44073FB602E4B01221A602C4B002224
:101CEC001A60294AFB681362FB6803F00103002B9E
:101CFC0014D0FFF72BFB38610AE0FFF727FB0246F5
:101D0C003B69D31A41F28832934201D9032336E05E
:101D1C001D4B1B6A03F00203002BEED01A4B1B6AFF
:101D2C0023F440727B685B68174913430B62FB7D9D
:101D3C00012B05D1144BDB69134A23F08053D3617B
:101D4C007B681B6803F00203002B08D00E4B5B680A
:101D5C0023F440427B689B680B4913434B607B68C0
:101D6C001B6803F01003002B08D0074B5B6823F4AF
:101D7C0080027B68DB68044913434B6000231846E0
:101D8C001837BD4680BD00BF0010024000700040F7
:101D9C004004424280B588B000AF786000237B617C
:101DAC000023FB6100233B610023FB600023BB612C
:101DBC007B68102B0AD07B68102B00F28A807B6822
:101DCC00012B45D07B68022B75D082E0464B5B68BB
:101DDC00FB60454B1B6803F08073002B7BD0FB68CA
:101DEC009B0C03F00F03414AD35C3B61FB6803F48B
:101DFC008033002B15D03C4B5B685B0C03F001036C
:101E0C003B4AD35C7B61FB6803F48033002B0DD021
:101E1C00384A7B69B2FBF3F23B6902FB03F3FB61CB
:101E2C0004E03B69344A02FB03F3FB612E4B5B6815
:101E3C0003F48003B3F5800F02D1FB69BB614AE068
:101E4C00FB695B002D4AA2FB03235B08BB6142E0EC
:101E5C00254B1B6AFB60FB6803F44073B3F5807F72
:101E6C0008D1FB6803F00203002B03D04FF40043AE
:101E7C00BB611FE0FB6803F44073B3F5007F09D12D
:101E8C00194B5B6A03F00203002B03D049F6404365
:101E9C00BB610FE0FB6803F44073B3F5407F1CD1CA
:101EAC00114B1B6803F40033002B16D04FF2244364
:101EBC00BB6112E011E0FFF755FE02460A4B5B686E
:101ECC009B0B03F0030301335B00B2FBF3F3BB6129
:101EDC0004E000BF02E000BF00E000BFBB69184691
:101EEC002037BD4680BD00BF00100240E4740008DE
:101EFC00F474000800127A0000093D00ABAAAAAAEB
:101F0C0080B48BB000AF7860396000237B62002313
:101F1C003B6269E101227B6A02FA03F3FB613B68D5
:101F2C001B68FA691340BB61BA69FB699A4240F0BD
:101F3C0058813B685B689A4A93425ED0984A9342B8
:101F4C0075D8984A934258D0964A93426FD8964A7D
:101F5C00934252D0944A934269D8944A93424CD0BB
:101F6C00924A934263D8924A934246D0904A934203
:101F7C005DD8122B2AD8122B59D801A252F823F073
:101F8C0007200008E11F0008F31F00083520000897
:101F9C003B2000083B2000083B2000083B200008A9
:101FAC003B2000083B2000083B2000083B20000899
:101FBC003B2000083B2000083B2000083B20000889
:101FCC003B200008E91F0008FD1F0008794A9342D6
:101FDC0013D02CE03B68DB683B6229E03B68DB6894
:101FEC0004333B6224E03B68DB6808333B621FE050
:101FFC003B68DB680C333B621AE03B689B68002B48
:10200C0002D104233B6213E03B689B68012B05D192
:10201C0008233B627B68FA691A6109E008233B627A
:10202C007B68FA695A6103E000233B6200E000BF61
:10203C00BB69FF2B01D87B6801E07B6804337B61B3
:10204C00BB69FF2B02D87B6A9B0002E07B6A083BD2
:10205C009B003B617B691A680F213B6901FA03F312
:10206C00DB431A40396A3B6901FA03F31A437B6973
:10207C001A603B685B6803F08053002B00F0B18062
:10208C004D4B9B694C4A43F0010393614A4B9B694E
:10209C0003F00103BB60BB68484A7B6A9B080233B0
:1020AC0052F82330FB607B6A03F003039B000F2282
:1020BC0002FA03F3DB43FA681340FB607B68404A87
:1020CC00934213D07B683F4A93420DD07B683E4AC3
:1020DC00934207D07B683D4A934201D1032306E02B
:1020EC00042304E0022302E0012300E000237A6AC7
:1020FC0002F0030292009340FA681343FB602F49ED
:10210C007B6A9B080233FA6841F823203B685B68C2
:10211C0003F48013002B06D02D4B9A682C49BB6915
:10212C0013438B6006E02A4B9A68BB69DB43284952
:10213C0013408B603B685B6803F40013002B06D0E4
:10214C00234BDA682249BB691343CB6006E0204B72
:10215C00DA68BB69DB431E491340CB603B685B68A4
:10216C0003F40033002B06D0194B5A681849BB698D
:10217C0013434B6006E0164B5A68BB69DB431449AA
:10218C0013404B603B685B6803F48033002B21D019
:10219C000F4B1A680E49BB6913430B6021E000BF5B
:1021AC00000032100000311000002210000021103D
:1021BC00000012100000111000100240000001403D
:1021CC0000080140000C01400010014000140140C7
:1021DC00000401400B4B1A68BB69DB4309491340EF
:1021EC000B607B6A01337B623B681A687B6A22FA5C
:1021FC0003F3002B7FF48EAE00BF00BF2C37BD461F
:10220C0080BC70470004014080B485B000AF78609A
:10221C000B467B807B689A687B881340002B02D02E
:10222C000123FB7301E00023FB73FB7B184614377F
:10223C00BD4680BC704780B483B000AF78600B465D
:10224C007B8013467B707B78002B03D07A887B686D
:10225C001A6103E07B881A047B681A6100BF0C3793
:10226C00BD4680BC7047000080B582B000AF03460D
:10227C00FB80084B5A69FB881340002B06D0054A9B
:10228C00FB885361FB88184603F0E0F800BF083761
:10229C00BD4680BD0004014080B485B000AF7860BD
:1022AC000023FB607B68002B01D1012343E07B689A
:1022BC001B681A46224B1344224AA2FB03231B0918
:1022CC009A007B681A647B681F4ADA637B68022277
:1022DC0083F821207B681B681B68FB60FB6823F478
:1022EC007F5323F03003FB607B685A687B689B68E4
:1022FC001A437B68DB681A437B681B691A437B684B
:10230C005B691A437B689B691A437B68DB691343DF
:10231C00FA681343FB607B681B68FA681A607B6879
:10232C0000229A637B68012283F821207B680022BB
:10233C0083F82020002318461437BD4680BC704714
:10234C00F8FFFDBFCDCCCCCC0000024080B586B0F0
:10235C0000AFF860B9607A603B600023FB75FB68E6
:10236C0093F82030012B01D102234BE0FB680122B2
:10237C0083F82020FB6893F82130DBB2012B3AD193
:10238C00FB68022283F82120FB6800229A63FB6819
:10239C001B681A68FB681B6822F001021A603B6814
:1023AC007A68B968F86800F0EBF9FB68DB6A002B17
:1023BC0008D0FB681B681A68FB681B6842F00E02A9
:1023CC001A600FE0FB681B681A68FB681B6822F038
:1023DC0004021A60FB681B681A68FB681B6842F0F1
:1023EC000A021A60FB681B681A68FB681B6842F0DB
:1023FC0001021A6005E0FB68002283F8202002230A
:10240C00FB75FB7D18461837BD4680BD80B485B082
:10241C0000AF78600023FB737B6893F82130DBB24C
:10242C00022B08D07B6804229A637B68002283F815
:10243C002020012320E07B681B681A687B681B68DE
:10244C0022F00E021A607B681B681A687B681B6896
:10245C0022F001021A607B681A6C7B68DB6B01212D
:10246C0001FA02F25A607B68012283F821207B6812
:10247C00002283F82020FB7B18461437BD4680BC15
:10248C007047000080B584B000AF78600023FB7308
:10249C007B6893F82130DBB2022B05D07B680422D9
:1024AC009A630123FB7351E07B681B681A687B6895
:1024BC001B6822F00E021A607B681B681A687B6826
:1024CC001B6822F001021A607B681B68224A934247
:1024DC0029D07B681B68214A934222D07B681B68F9
:1024EC001F4A93421AD07B681B681E4A934212D033
:1024FC007B681B681C4A93420AD07B681B681B4A8A
:10250C00934202D14FF480130EE04FF080730BE036
:10251C004FF4803308E04FF4805305E04FF48073A0
:10252C0002E0102300E00123114A53607B68012272
:10253C0083F821207B68002283F820207B685B6B6A
:10254C00002B03D07B685B6B78689847FB7B184645
:10255C001037BD4680BD00BF080002401C00024081
:10256C003000024044000240580002406C0002401F
:10257C000000024080B584B000AF78607B68DB6BF4
:10258C001B68FB607B681B681B68BB607B681B6CF3
:10259C0004229A40FB681340002B4FD0BB6803F019
:1025AC000403002B4AD07B681B681B6803F02003D4
:1025BC00002B07D17B681B681A687B681B6822F0AC
:1025CC0004021A607B681B68664A934229D07B68B8
:1025DC001B68654A934222D07B681B68634A93420E
:1025EC001AD07B681B68624A934212D07B681B68C6
:1025FC00604A93420AD07B681B685F4A934202D1BF
:10260C004FF480030EE04FF080630BE04FF4802317
:10261C0008E04FF4804305E04FF4806302E0402370
:10262C0000E00423554A53607B68DB6A002B00F002
:10263C0094807B68DB6A786898478EE07B681B6CBB
:10264C0002229A40FB681340002B56D0BB6803F063
:10265C000203002B51D07B681B681B6803F020031E
:10266C00002B0BD17B681B681A687B681B6822F0F7
:10267C000A021A607B68012283F821207B681B68A0
:10268C00384A934229D07B681B68374A934222D040
:10269C007B681B68354A93421AD07B681B68344AA6
:1026AC00934212D07B681B68324A93420AD07B68F3
:1026BC001B68314A934202D14FF400130EE04FF0E5
:1026CC0000730BE04FF4003308E04FF4005305E0C7
:1026DC004FF4007302E0202300E00223274A5360EA
:1026EC007B68002283F820207B689B6A002B34D007
:1026FC007B689B6A786898472FE07B681B6C082284
:10270C009A40FB681340002B28D0BB6803F00803E9
:10271C00002B23D07B681B681A687B681B6822F02F
:10272C000E021A607B681A6C7B68DB6B012101FA64
:10273C0002F25A607B6801229A637B68012283F85B
:10274C0021207B68002283F820207B681B6B002BE8
:10275C0004D07B681B6B7868984700BF00BF1037AC
:10276C00BD4680BD080002401C0002403000024003
:10277C0044000240580002406C000240000002403D
:10278C0080B485B000AFF860B9607A603B60FB68DC
:10279C001A6CFB68DB6B012101FA02F25A60FB68D0
:1027AC001B683A685A60FB685B68102B08D1FB68A1
:1027BC001B687A689A60FB681B68BA68DA6007E085
:1027CC00FB681B68BA689A60FB681B687A68DA60F9
:1027DC0000BF1437BD4680BC7047000080B485B084
:1027EC0000AF78607B6803F00703FB600C4BDB6881
:1027FC00BB60BA684FF6FF031340BB60FB681A025C
:10280C00BB68134343F0BF6343F40033BB60044A1B
:10281C00BB68D36000BF1437BD4680BC704700BF97
:10282C0000ED00E080B400AF044BDB681B0A03F042
:10283C0007031846BD4680BC704700BF00ED00E0A2
:10284C0080B483B000AF0346FB7197F90730002BBF
:10285C000BDBFB7903F01F02064997F907305B0984
:10286C00012000FA02F241F8232000BF0C37BD46CC
:10287C0080BC704700E100E080B483B000AF034639
:10288C003960FB7197F90730002B0ADB3B68DAB231
:10289C000C4997F907301201D2B20B4483F800238C
:1028AC000AE03B68DAB20849FB7903F00F03043BFA
:1028BC001201D2B20B441A7600BF0C37BD4680BC55
:1028CC00704700BF00E100E000ED00E080B489B08B
:1028DC0000AFF860B9607A60FB6803F00703FB6136
:1028EC00FB69C3F10703042B28BF0423BB61FB69FD
:1028FC000433062B02D9FB69033B00E000237B6108
:10290C004FF0FF32BB6902FA03F3DA43BB681A409B
:10291C007B699A404FF0FF317B6901FA03F3D9438D
:10292C007B680B40134318462437BD4680BC704768
:10293C0080B582B000AF78607868FFF74FFF00BFBA
:10294C000837BD4680BD80B586B000AF0346B96080
:10295C007A60FB7300237B61FFF764FF78617A6810
:10296C00B9687869FFF7B2FF024697F90F30114644
:10297C001846FFF781FF00BF1837BD4680BD80B5F4
:10298C0082B000AF0346FB7197F907301846FFF78A
:10299C0057FF00BF0837BD4680BD000080B400AFB4
:1029AC00034B01221A6000BFBD4680BC704700BFBC
:1029BC0020000E4280B400AF084B1B68074A43F05E
:1029CC0002031360064B1B69054A43F004031361B1
:1029DC0030BF00BFBD4680BC704700BF00700040D8
:1029EC0000ED00E0F0B587B000AFF860B960C7E962
:1029FC0000230123FB750023BB7500237B752F4B34
:102A0C001B7E012B01D1022354E02C4B01221A76A0
:102A1C004CF2503000F0A8F80346FB75FB7D002B00
:102A2C0044D1FB68012B02D101237B7507E0FB68C5
:102A3C00022B02D102237B7501E004237B7500235A
:102A4C00BB752DE0BB7D5A00BB6802EB030CBB7D54
:102A5C001901D7E90023C1F12006A1F1200022FAC7
:102A6C0001F403FA06F6344323FA00F0044323FA84
:102A7C0001F5A3B21946604600F05AF84CF25030FA
:102A8C0000F072F80346FB750D4B1B690C4A23F0E2
:102A9C0001031361FB7D002B07D1BB7D0133BB759B
:102AAC00BA7D7B7D9A42CDD300E000BF034B002260
:102ABC001A76FB7D18461C37BD46F0BD98000020E9
:102ACC000020024080B483B000AF0023FB710D4B9B
:102ADC001B6903F08003002B0DD00A4B0A4A5A6085
:102AEC00084B0A4A5A60074B1B6903F08003002B02
:102AFC0001D00123FB71FB7918460C37BD4680BC15
:102B0C00704700BF0020024023016745AB89EFCD21
:102B1C0080B400AF054B1B69044A43F0800313617A
:102B2C0000231846BD4680BC704700BF0020024001
:102B3C0080B483B000AF78600B467B80084B0022DA
:102B4C00DA61084B1B69074A43F0010313617B6888
:102B5C007A881A8000BF0C37BD4680BC704700BF16
:102B6C00980000200020024080B584B000AF78604F
:102B7C00FEF7ECFBF86010E07B68B3F1FF3F0CD084
:102B8C007B68002B07D0FEF7E1FB0246FB68D31AEB
:102B9C007A689A4201D2032325E0154BDB6803F0D7
:102BAC000103002BE8D1124BDB6803F02003002B50
:102BBC0002D00F4B2022DA600D4BDB6803F01003C0
:102BCC00002B0BD10A4BDB6903F00103002B05D161
:102BDC00074BDB6803F00403002B03D000F00AF86A
:102BEC00012300E0002318461037BD4680BD00BF0E
:102BFC000020024080B483B000AF00237B60234BE5
:102C0C00DB6803F01003002B09D0214BDB6943F088
:102C1C0002031F4AD3617B6843F010037B601B4B9C
:102C2C00DB6803F00403002B09D0194BDB6943F07C
:102C3C000103174AD3617B6843F004037B60134B99
:102C4C00DB6903F00103002B0BD0114BDB6943F064
:102C5C0004030F4AD3610D4BDB690C4A23F00103CB
:102C6C00D3617B6840F20112934206D1074BDB69BA
:102C7C00064A23F00103D36102E0044A7B68D36067
:102C8C0000BF0C37BD4680BC704700BF002002401F
:102C9C009800002080B584B000AF786039600123C3
:102CAC00FB730023BB602F4B1B7E012B01D1022336
:102CBC0053E02C4B01221A767B681B68022B16D131
:102CCC004CF25030FFF750FF0346002B41D101204E
:102CDC0000F04CF84CF25030FFF746FF0346FB7304
:102CEC00214B1B69204A23F00403136131E04CF2A1
:102CFC005030FFF739FF0346002B2AD13B684FF0C9
:102D0C00FF321A607B689B68BB6019E0B86800F002
:102D1C0049F84CF25030FFF727FF0346FB73124B78
:102D2C001B69114A23F002031361FB7B002B03D0B8
:102D3C003B68BA681A600CE0BB6803F58063BB6043
:102D4C007B68DB689A027B689B681344BA689A427A
:102D5C00DCD3044B00221A76FB7B18461037BD4699
:102D6C0080BD00BF980000200020024080B483B0DA
:102D7C0000AF7860094B0022DA61094B1B69084AE5
:102D8C0043F004031361064B1B69054A43F04003EF
:102D9C00136100BF0C37BD4680BC70479800002003
:102DAC000020024080B483B000AF78600B4B00224F
:102DBC00DA610B4B1B690A4A43F002031361084AA0
:102DCC007B685361064B1B69054A43F04003136152
:102DDC0000BF0C37BD4680BC704700BF9800002078
:102DEC000020024080B582B000AF78607B68002B79
:102DFC0001D1012342E07B6893F84130DBB2002B18
:102E0C0006D17B68002283F84020786802F0D8FB5A
:102E1C007B68242283F841207B681B68DA687B6816
:102E2C001B6822F40052DA60786800F0CFFF7B68F0
:102E3C001B681A697B681B6822F490421A617B68D4
:102E4C001B685A697B681B6822F02A025A617B68EE
:102E5C001B68DA687B681B6842F40052DA607B6896
:102E6C0000225A647B68202283F841207B68202250
:102E7C0083F842207B6800225A63002318460837E7
:102E8C00BD4680BD80B58AB002AFF860B9603B60CA
:102E9C001346FB8000237B61FB6893F84130DBB267
:102EAC00202B75D1BB68002B02D0FB88002B01D1E5
:102EBC0001236EE0FB6800225A64FB68212283F830
:102ECC004120FEF743FA7861FB68FA889A84FB6824
:102EDC00FA88DA84FB689B68B3F5805F08D1FB68DD
:102EEC001B69002B04D10023FB61BB68BB6103E0B1
:102EFC00BB68FB610023BB612EE03B6800937B69E0
:102F0C0000228021F86800F0ACFC0346002B05D0B1
:102F1C00FB68202283F8412003233AE0FB69002B55
:102F2C000BD1BB691B881A46FB681B68C2F30802ED
:102F3C005A60BB690233BB6107E0FB691A78FB6816
:102F4C001B685A60FB690133FB61FB68DB8C9BB22D
:102F5C00013B9AB2FB68DA84FB68DB8C9BB2002BDA
:102F6C00CBD13B6800937B6900224021F86800F0CC
:102F7C0078FC0346002B05D0FB68202283F8412007
:102F8C00032306E0FB68202283F84120002300E0A5
:102F9C00022318462037BD4680BD80B584B000AFF3
:102FAC00F860B9601346FB80FB6893F84230DBB2E3
:102FBC00202B12D1BB68002B02D0FB88002B01D137
:102FCC0001230BE0FB6800221A63FB881A46B968E0
:102FDC00F86800F09FFC034600E002231846103707
:102FEC00BD4680BD80B590B000AF78600023FB6318
:102FFC007B681B685B6903F08003002B14BF012303
:10300C000023DBB2FB637B6893F84130DBB2212BEE
:10301C0028D1FB6B002B25D07B681B6814337B629B
:10302C007B6A53E8003F3B623B6A23F08003BB633F
:10303C007B681B681433BA6B3A63FB62F96A3A6BB0
:10304C0041E80023BB62BB6A002BE5D17B689B6B1C
:10305C00002B04D07B689B6B1846FFF7D7F9786878
:10306C0000F0F2FC7B681B685B6903F04003002BEB
:10307C0014BF01230023DBB2FB637B6893F842305F
:10308C00DBB2222B28D1FB6B002B25D07B681B6875
:10309C0014333B613B6953E8003FFB60FB6823F052
:1030AC0040037B637B681B6814337A6BFA61BB61EA
:1030BC00B969FA6941E800237B617B69002BE5D192
:1030CC007B68DB6B002B04D07B68DB6B1846FFF74F
:1030DC009DF9786800F0DFFC002318464037BD46A8
:1030EC0080BD000080B5BAB000AF78607B681B680B
:1030FC001B68C7F8E4307B681B68DB68C7F8E030F6
:10310C007B681B685B69C7F8DC300023C7F8D830D4
:10311C000023C7F8D430D7F8E43003F00F03C7F816
:10312C00D830D7F8D830002B0FD1D7F8E43003F0D3
:10313C002003002B09D0D7F8E03003F02003002B3C
:10314C0003D0786800F084FD5BE2D7F8D830002B10
:10315C0000F0DE80D7F8DC3003F00103002B06D141
:10316C00D7F8E03003F49073002B00F0D180D7F83F
:10317C00E43003F00103002B0BD0D7F8E03003F45C
:10318C008073002B05D07B685B6C43F001027B687D
:10319C005A64D7F8E43003F00403002B0BD0D7F8B3
:1031AC00DC3003F00103002B05D07B685B6C43F033
:1031BC0002027B685A64D7F8E43003F00203002B58
:1031CC000BD0D7F8DC3003F00103002B05D07B6863
:1031DC005B6C43F004027B685A64D7F8E43003F06C
:1031EC000803002B11D0D7F8E03003F02003002B9C
:1031FC0005D1D7F8DC3003F00103002B05D07B6838
:10320C005B6C43F008027B685A647B685B6C002B38
:10321C0000F0F281D7F8E43003F02003002B08D043
:10322C00D7F8E03003F02003002B02D0786800F0D0
:10323C000FFD7B681B685B6903F04003002B14BF18
:10324C0001230023DBB2C7F8D4307B685B6C03F03E
:10325C000803002B03D1D7F8D430002B4FD078685B
:10326C0000F019FC7B681B685B6903F04003002BC2
:10327C0041D07B681B681433C7F89C30D7F89C305E
:10328C0053E8003FC7F89830D7F8983023F0400344
:10329C00C7F8D0307B681B681433D7F8D020C7F838
:1032AC00A820C7F8A430D7F8A410D7F8A82041E874
:1032BC000023C7F8A030D7F8A030002BD9D17B68F9
:1032CC00DB6B002B13D07B68DB6B7E4A5A637B680D
:1032DC00DB6B1846FFF7D6F80346002B16D07B683D
:1032EC00DB6B5B6B7A68D26B104698470EE07868A4
:1032FC0000F0A5F90AE0786800F0A1F906E078681A
:10330C0000F09DF97B6800225A6475E100BF73E1FF
:10331C007B681B6B012B40F04F81D7F8E43003F036
:10332C001003002B00F04881D7F8E03003F01003B5
:10333C00002B00F041810023BB607B681B681B687D
:10334C00BB607B681B685B68BB60BB687B681B6889
:10335C005B6903F04003002B00F0B6807B68DB6BED
:10336C001B685B68A7F8BE30B7F8BE30002B00F0C6
:10337C0045817B689B8DB7F8BE209A4280F03E81D8
:10338C007B68B7F8BE20DA857B68DB6B9B69202BEA
:10339C0000F088807B681B680C33C7F88830D7F83E
:1033AC00883053E8003FC7F88430D7F8843023F4D2
:1033BC008073C7F8B8307B681B680C33D7F8B8201B
:1033CC00C7F89420C7F89030D7F89010D7F894200D
:1033DC0041E80023C7F88C30D7F88C30002BD9D1BA
:1033EC007B681B6814337B677B6F53E8003F3B673C
:1033FC003B6F23F00103C7F8B4307B681B681433B0
:10340C00D7F8B420C7F88020FB67F96FD7F8802075
:10341C0041E80023BB67BB6F002BE1D17B681B68C5
:10342C0014333B663B6E53E8003FFB65FB6D23F0AA
:10343C004003C7F8B0307B681B681433D7F8B02052
:10344C00FA66BB66B96EFA6E41E800237B667B6E4A
:10345C00002BE3D17B68202283F842207B6800227A
:10346C001A637B681B680C33FB64FB6C53E8003FEE
:10347C00BB64BB6C23F01003C7F8AC307B681B68D3
:10348C000C33D7F8AC20BA657B65796DBA6D41E821
:10349C0000233B653B6D002BE3D17B68DB6B18464F
:1034AC00FEF7B4FF7B6802225A637B689A8D7B68B7
:1034BC00DB8D9BB2D31A9BB21946786800F0C8F822
:1034CC009CE000BF673B00087B689A8D7B68DB8DB6
:1034DC009BB2D31AA7F8CE307B68DB8D9BB2002B46
:1034EC0000F08E80B7F8CE30002B00F089807B681E
:1034FC001B680C33BB63BB6B53E8003F7B637B6B7C
:10350C0023F49073C7F8C8307B681B680C33D7F86A
:10351C00C8207A643B64396C7A6C41E80023FB6305
:10352C00FB6B002BE3D17B681B6814337B627B6ADB
:10353C0053E8003F3B623B6A23F00103C7F8C430F9
:10354C007B681B681433D7F8C4203A63FB62F96AB2
:10355C003A6B41E80023BB62BB6A002BE3D17B686A
:10356C00202283F842207B6800221A637B681B6848
:10357C000C333B613B6953E8003FFB60FB6823F075
:10358C001003C7F8C0307B681B680C33D7F8C02019
:10359C00FA61BB61B969FA6941E800237B617B6917
:1035AC00002BE3D17B6802225A63B7F8CE30194660
:1035BC00786800F04DF823E0D7F8E43003F080038E
:1035CC00002B09D0D7F8E03003F08003002B03D098
:1035DC00786800F0D6FA14E0D7F8E43003F0400332
:1035EC00002B0ED0D7F8E03003F04003002B08D0AE
:1035FC00786800F015FB04E000BF02E000BF00E0BB
:10360C0000BFE837BD4680BD80B483B000AF7860A2
:10361C0000BF0C37BD4680BC704780B483B000AF90
:10362C00786000BF0C37BD4680BC704780B483B057
:10363C0000AF786000BF0C37BD4680BC704780B4CB
:10364C0083B000AF786000BF0C37BD4680BC7047BC
:10365C0080B483B000AF78600B467B8000BF0C3722
:10366C00BD4680BC704780B59CB000AF78607B686D
:10367C005B6AFB667B681B681B6803F02003002BEE
:10368C0072D1FB6E0022DA85FB6E1B680C33FB6477
:10369C00FB6C53E8003FBB64BB6C23F48073BB66CC
:1036AC00FB6E1B680C33BA6EBA657B65796DBA6DAF
:1036BC0041E800233B653B6D002BE5D1FB6E1B689D
:1036CC001433BB63BB6B53E8003F7B637B6B23F012
:1036DC0001037B66FB6E1B6814337A6E7A643B6461
:1036EC00396C7A6C41E80023FB63FB6B002BE5D152
:1036FC00FB6E1B6814337B627B6A53E8003F3B62B2
:10370C003B6A23F040033B66FB6E1B6814333A6E36
:10371C003A63FB62F96A3A6B41E80023BB62BB6A0D
:10372C00002BE5D1FB6E202283F84220FB6E1B6B35
:10373C00012B19D1FB6E1B680C333B613B6953E8C1
:10374C00003FFB60FB6823F01003FB65FB6E1B68FE
:10375C000C33FA6DFA61BB61B969FA6941E800236F
:10376C007B617B69002BE5D1FB6E00225A63FB6EFB
:10377C001B6B012B06D1FB6E9B8D1946F86EFFF768
:10378C0067FF02E0F86EFFF748FF00BF7037BD46D9
:10379C0080BD80B584B000AF78607B685B6AFB60ED
:1037AC00FB6801225A63FB681B6B012B08D1FB6879
:1037BC009B8D5B089BB21946F868FFF749FF02E046
:1037CC00F868FFF733FF00BF1037BD4680BD80B5EA
:1037DC0084B000AF78600023FB607B685B6ABB60E1
:1037EC00BB681B685B6903F08003002B14BF0123CB
:1037FC000023DBB2FB60BB6893F84130DBB2212BBA
:10380C0008D1FB68002B05D0BB680022DA84B868AD
:10381C0000F01AF9BB681B685B6903F04003002BCE
:10382C0014BF01230023DBB2FB60BB6893F842306A
:10383C00DBB2222B08D1FB68002B05D0BB68002221
:10384C00DA85B86800F027F9BB685B6C43F01002AE
:10385C00BB685A64B868FFF7F2FE00BF1037BD466C
:10386C0080BD80B586B000AFF860B9603B60134690
:10387C00FB713BE03B6AB3F1FF3F37D0FDF766FDD0
:10388C0002463B68D31A3A6A9A4202D33B6A002B2F
:10389C0001D103233AE0FB681B68DB6803F00403E7
:1038AC00002B23D0BB68802B20D0BB68402B1DD0B5
:1038BC00FB681B681B6803F00803082B16D1002358
:1038CC007B61FB681B681B687B61FB681B685B6822
:1038DC007B617B69F86800F0DEF8FB6808225A64AB
:1038EC00FB68002283F8402001230FE0FB681B6873
:1038FC001A68BB681340BA689A420CBF01230023B4
:10390C00DBB21A46FB799A42B4D00023184618371A
:10391C00BD4680BD80B598B000AFF860B960134665
:10392C00FB80BA68FB689A62FB68FA889A85FB6828
:10393C0000225A64FB68222283F84220FB68DB6B6E
:10394C003E4A9A62FB68DB6B3D4ADA62FB68DB6BD2
:10395C003C4A1A63FB68DB6B00225A6307F10803CD
:10396C00FB65FB68D86BFB681B6804331946FB6D61
:10397C001A68FB88FEF7EAFC00233B61FB681B68B6
:10398C001B683B61FB681B685B683B613B69FB68C0
:10399C001B69002B19D0FB681B680C333B643B6C18
:1039AC0053E8003FFB63FB6B43F48073BB65FB6820
:1039BC001B680C33BA6DFA64BB64B96CFA6C41E8E1
:1039CC0000237B647B6C002BE5D1FB681B681433F4
:1039DC00FB62FB6A53E8003FBB62BB6A43F0010326
:1039EC007B65FB681B6814337A6DBA637B63796BF8
:1039FC00BA6B41E800233B633B6B002BE5D1FB68C2
:103A0C001B681433BB61BB6953E8003F7B617B6966
:103A1C0043F040033B65FB681B6814333A6D7A62D4
:103A2C003B62396A7A6A41E80023FB61FB69002B2F
:103A3C00E5D1002318466037BD4680BD73360008BB
:103A4C009F370008DB37000880B489B000AF78607E
:103A5C007B681B680C33FB60FB6853E8003FBB6062
:103A6C00BB6823F0C003FB617B681B680C33FA69ED
:103A7C00BA617B617969BA6941E800233B613B69B2
:103A8C00002BE5D17B68202283F8412000BF24372E
:103A9C00BD4680BC704780B495B000AF78607B6841
:103AAC001B680C337B637B6B53E8003F3B633B6BC6
:103ABC0023F49073FB647B681B680C33FA6C3A64D8
:103ACC00FB63F96B3A6C41E80023BB63BB6B002BC7
:103ADC00E5D17B681B6814333B623B6A53E8003FBB
:103AEC00FB61FB6923F00103BB647B681B68143327
:103AFC00BA6CFA62BB62B96AFA6A41E800237B626B
:103B0C007B6A002BE5D17B681B6B012B19D17B6881
:103B1C001B680C33FB60FB6853E8003FBB60BB6861
:103B2C0023F010037B647B681B680C337A6CBA61DE
:103B3C007B617969BA6941E800233B613B69002BE1
:103B4C00E5D17B68202283F842207B6800221A632F
:103B5C0000BF5437BD4680BC704780B584B000AF01
:103B6C0078607B685B6AFB60FB680022DA85FB6827
:103B7C000022DA84F868FFF762FD00BF1037BD46FB
:103B8C0080BD80B485B000AF78607B6893F841301D
:103B9C00DBB2212B3ED17B689B68B3F5805F14D1DF
:103BAC007B681B69002B10D17B681B6AFB60FB6870
:103BBC001B881A467B681B68C2F308025A607B6834
:103BCC001B6A9A1C7B681A6208E07B681B6A591C8A
:103BDC007A6811621A787B681B685A607B68DB8C88
:103BEC009BB2013B9BB27A681946D184002B0FD152
:103BFC007B681B68DA687B681B6822F08002DA60DD
:103C0C007B681B68DA687B681B6842F04002DA60EC
:103C1C00002300E0022318461437BD4680BC7047D1
:103C2C0080B582B000AF78607B681B68DA687B680F
:103C3C001B6822F04002DA607B68202283F8412066
:103C4C007868FFF7E1FC002318460837BD4680BDB5
:103C5C0080B58CB000AF78607B6893F84230DBB2F3
:103C6C00222B40F0AE807B689B68B3F5805F17D148
:103C7C007B681B69002B13D10023FB627B689B6A5A
:103C8C00BB627B681B685B689BB2C3F308039AB288
:103C9C00BB6A1A807B689B6A9A1C7B689A6226E0D6
:103CAC007B689B6AFB620023BB627B689B68B3F5F5
:103CBC00805F07D07B689B68002B0AD17B681B69EF
:103CCC00002B06D17B681B685B68DAB2FB6A1A7042
:103CDC0008E07B681B685B68DBB203F07F03DAB239
:103CEC00FB6A1A707B689B6A5A1C7B689A627B68B9
:103CFC00DB8D9BB2013B9BB27A681946D185002BB8
:103D0C005DD17B681B68DA687B681B6822F0200237
:103D1C00DA607B681B68DA687B681B6822F4807247
:103D2C00DA607B681B685A697B681B6822F00102A9
:103D3C005A617B68202283F842207B6800225A63F8
:103D4C007B681B6B012B35D17B6800221A637B6867
:103D5C001B680C337B617B6953E8003F3B613B691B
:103D6C0023F010037B627B681B680C337A6A3A621F
:103D7C00FB61F9693A6A41E80023BB61BB69002B1E
:103D8C00E5D17B681B681B6803F01003102B0AD16C
:103D9C000023FB607B681B681B68FB607B681B68EF
:103DAC005B68FB60FB687B689B8D19467868FFF746
:103DBC004FFC02E07868FFF730FC002302E00023A0
:103DCC0000E0022318463037BD4680BD80B584B074
:103DDC0000AF78607B681B681B6923F440517B68DB
:103DEC00DA687B681B680A431A617B689A687B688F
:103DFC001B691A437B685B691343BB607B681B6858
:103E0C00DB6823F4B05323F00C037A681268B968AA
:103E1C000B43D3607B681B685B6923F440717B6840
:103E2C009A697B681B680A435A617B681B682C4A39
:103E3C00934203D1FDF796FEF86002E0FDF77EFE9B
:103E4C00F860FA6813469B0013449A001A447B6886
:103E5C005B689B00B2FBF3F3224AA2FB03235B09D2
:103E6C001901FA6813469B0013449A001A447B68A4
:103E7C005B689B00B2FBF3F21A4BA3FB02035B09DA
:103E8C00642000FB03F3D31A1B013233154AA2FB47
:103E9C0003235B0903F0F0031944FA6813469B00F3
:103EAC0013449A001A447B685B689B00B2FBF3F2E4
:103EBC000C4BA3FB02035B09642000FB03F3D31A36
:103ECC001B013233074AA2FB03235B0903F00F02E9
:103EDC007B681B680A449A6000BF1037BD4680BDE2
:103EEC00003801401F85EB5180B500AF4FF0FF3318
:103EFC00092203490348FEF7C5FF00BF80BD00BF80
:103F0C00BC7000085404002080B500AF4FF0FF33A4
:103F1C000F2203490348FEF7B5FF00BF80BD00BF69
:103F2C00C87000085404002080B500AF4FF0FF3378
:103F3C00082203490348FEF7A5FF00BF80BD00BF60
:103F4C00D87000085404002080B500AF4FF0FF3348
:103F5C00082203490348FEF795FF00BF80BD00BF50
:103F6C00E47000085404002080B500AF4FF0FF331C
:103F7C000E2203490348FEF785FF00BF80BD00BF3A
:103F8C00F47000085404002080B500AF00224FF4F8
:103F9C0000410248FEF74FF900BF80BD0008014008
:103FAC0090B583B000AF0346FB71FB79002B1CD09E
:103FBC00FB79032B19D8FB790E4A52F82330002BCE
:103FCC0013D0FB790B4A52F82340FB79094A52F87B
:103FDC0023301846FCF7B4F803469AB24FF0FF337F
:103FEC0021460548FEF74EFF00E000BF0C37BD46EA
:103FFC0090BD00BF0C0000200C04002080B58AB0DE
:10400C0000AF104B1B791BB21B021AB20D4B5B7924
:10401C001BB213431BB2FB84FA8C3B1D0A49184696
:10402C0001F03EFF3B1D1846FCF78AF803469AB296
:10403C00391D4FF0FF330548FEF724FF00BF28372A
:10404C00BD4680BDB8000020047100080C0400209F
:10405C0080B584B000AF134801F01AFF55233B71B3
:10406C00AA237B710123BB710F4B9B78FB710E4B09
:10407C00DB783B720C4B5B787B720B4B1B79BB7206
:10408C00094B5B79FB72FF233B73EE237B73391D6A
:10409C004FF0FF330A220548FEF7F4FE00BF10373D
:1040AC00BD4680BD18710008B80000200C0400202B
:1040BC0080B586B000AF78600B46FB70164801F0F7
:1040CC00E7FE55233B72AA237B720223BB72134B70
:1040DC009B78FB72114BDB783B737A6807F10D030D
:1040EC001168526819605A607B7B002B01D1FF2349
:1040FC003B75FB787B75FF23BB75EE23FB7507F1D6
:10410C0008014FF0FF3310220548FEF7BBFE00BF3D
:10411C001837BD4680BD00BF2C710008B8000020C8
:10412C000C04002080B500AF184801F0B1FE184B0C
:10413C0001229A74174B5B79002B03D1144B01228B
:10414C00DA7403E0134B5A79114BDA74114B9B79E7
:10415C001B02104AD2791343002B0DD00D4B9B79C7
:10416C001BB21B021AB20B4BDB791BB213431BB2F3
:10417C009AB2074B1A8206E0074801F089FE044BFD
:10418C004FF4FA721A8200BF80BD00BF6071000844
:10419C00B8000020400500208471000880B500AFF5
:1041AC00184801F075FE184B1A7A184B1A71164BF9
:1041BC005A7A164B5A71144B5B79032B06D0032B8E
:1041CC0010DC012B0AD0022B04D00BE00F4B032286
:1041DC005A7014E00D4B02225A7010E00B4B012266
:1041EC005A700CE00A4801F053FE084BFF221A717A
:1041FC00064BFF225A71054B03225A7000BF00BFB9
:10420C0080BD00BFB071000840050020B800002040
:10421C00D871000880B582B000AF144801F038FEA8
:10422C00134B5B791A04124B9B791B021343104AF4
:10423C00D27913437B607B68002B03D07B680D4ADB
:10424C00934207D90C4801F023FE0C4B40F6B832D0
:10425C00DA6007E0094A7B68D3607968084801F0A6
:10426C00AFFD00BF00BF0837BD4680BD047200081B
:10427C00400500207F51010024720008B800002086
:10428C004C72000880B584B000AF134801F000FEFA
:10429C0055233B71AA237B710123BB710F4B9B7878
:1042AC00FB710E4BDB783B720C4B5B787B720B4BD0
:1042BC001B79BB72094B5B79FB72FF233B73EE23BB
:1042CC007B73391D4FF0FF330A220548FEF7DAFDE8
:1042DC0000BF1037BD4680BD70720008B8000020CA
:1042EC000C04002080B584B000AF134801F0D0FD61
:1042FC0055233B71AA237B710523BB710F4B9B7814
:10430C00FB710E4BDB783B720C4B5B787B720B4B6F
:10431C001B79BB72094B5B79FB72FF233B73EE235A
:10432C007B73391D4FF0FF330A220548FEF7AAFDB7
:10433C0000BF1037BD4680BD18710008B8000020C2
:10434C000C04002080B500AF1E4B9B78033B072B61
:10435C0031D801A252F823F085430008C34300086A
:10436C009D430008C343000891430008A94300087B
:10437C00C3430008B5430008FFF7D4FE124B2322B9
:10438C001A721CE0FFF70AFF0F4B27221A7216E075
:10439C00FFF740FF0C4B25221A7210E0FFF772FF5B
:1043AC00094B28221A720AE0074B01221A70064B9D
:1043BC0000221A7203E0044B00221A7200BF00BFE5
:1043CC0080BD00BF40050020B800002080B58AB039
:1043DC0000AF78607B68002B03D07B683B4A93422C
:1043EC0003D93B4801F054FD6DE007F1180300229E
:1043FC0019463848FCF714FA07F114030022194641
:10440C003448FCF79BFB3B7E1A464FF4616303FB7D
:10441C0002F27B7E19460B461B015B1A9B00134470
:10442C00BA7E13443B623A6A7B6813447B627B6AB4
:10443C00264A934205D97B6AA3F5A833A3F5C0732A
:10444C007B627B6A244AA2FB0323DB0AFB777A6A32
:10445C00214BA3FB0213DB0A4FF4616101FB03F355
:10446C00D31A1E4AA2FB03235B09BB77796A1B4B49
:10447C00A3FB01235A0913461B019B1A9B00CA1A62
:10448C0013467B7707F10C0300221A605A60FB7FFE
:10449C003B73BB7F7B737B7FBB7300233B6107F15B
:1044AC000C03002219460B48FCF79CFB0346002B1F
:1044BC0001D000F03BFE0A4B1B68094A43F0040391
:1044CC001360FEF777FA2837BD4680BD7F51010097
:1044DC00CC720008B0030020C5B3A29189888888EB
:1044EC000070004080B483B000AF78607B6800221D
:1044FC00A3F868217B680022A3F86A2100BF0C375F
:10450C00BD4680BC704780B483B000AF78607B68D8
:10451C00B3F868319AB27B68B3F86A319BB29A42AD
:10452C000CBF01230023DBB218460C37BD4680BC00
:10453C007047000080B483B000AF78607B68B3F83C
:10454C006A319BB25A1C0D4B83FB02131344191195
:10455C00D317C91A0B461B015B1A5B00D11A7B6877
:10456C00B3F868319BB299420CBF01230023DBB234
:10457C0018460C37BD4680BC704700BF89888888B8
:10458C0080B582B000AF786039607868FFF7D2FFF1
:10459C000346002B02D04FF0FF3325E07B68B3F8C5
:1045AC006A319BB21A4613465B0013449B007A682F
:1045BC0013440C223968184601F023FE7B68B3F8CB
:1045CC006A319BB25A1C0A4B83FB02131344191118
:1045DC00D317C91A0B461B015B1A5B00D11A8AB29E
:1045EC007B68A3F86A21002318460837BD4680BDB6
:1045FC008988888880B582B000AF78603960786827
:10460C00FFF781FF0346002B02D04FF0FF3325E06C
:10461C007B68B3F868319BB21A4613465B001344AF
:10462C009B007A6813440C221946386801F0E9FDA6
:10463C007B68B3F868319BB25A1C0A4B83FB02139C
:10464C0013441911D317C91A0B461B015B1A5B00D3
:10465C00D11A8AB27B68A3F8682100231846083760
:10466C00BD4680BD8988888880B584B000AF7860ED
:10467C007B68DBB2FB7307F10F014FF0FF330122B4
:10468C000348FEF7FFFB7B6818461037BD4680BD1C
:10469C00C403002080B500AF1248FFF723FF124877
:1046AC00FFF720FF114B00221A70104B03225A7097
:1046BC000E4BFE229A700D4BEF22DA700B4B002240
:1046CC009A710A4BFF221A71084BFF225A71074B41
:1046DC000022DA71054B0122DA71044B00221A72A6
:1046EC0000BF80BDCC00002038020020B8000020A4
:1046FC0080B500AF01224FF480710548FDF79BFD9A
:10470C00012208210348FDF796FD00BF80BD00BFC4
:10471C0000080140000C0140B0B588B000AF034662
:10472C000A46FB711346BB71FEF7CCF90023BB6044
:10473C000023FB60124B7B610123BB6107F1080274
:10474C0007F10C0311461846FEF7A4FAFB791BB2CD
:10475C001B021AB2BB791BB213431BB2FB83FB8B3C
:10476C0000221C46154622462B4605490120FEF721
:10477C0039F9FEF7CDF900BF2037BD46B0BD00BFFB
:10478C0000FC000880B485B000AF78603960094B3C
:10479C001B88FB81FB891B0A9BB2DAB27B681A70FF
:1047AC00FB89DAB23B681A7000BF1437BD4680BC77
:1047BC00704700BF00FC000880B487B000AF786081
:1047CC0039607B681B781A464FF4616303FB02F275
:1047DC007B685B7819460B461B015B1A9B001344E4
:1047EC007A68927813443B613B681B781A464FF405
:1047FC00616303FB02F23B685B7819460B461B01B5
:10480C005B1A9B0013443A6892781344FB60FA6875
:10481C003B69D31A7B617B69002B05DA7B6903F555
:10482C00A83303F5C0737B617B6918461C37BD4602
:10483C0080BC704780B586B000AFF860B9607A6014
:10484C0007F1100300210A461A800A469A7007F1F4
:10485C00100300221946F868FBF7E2FF07F110037A
:10486C001946B868FFF7A8FF78617B697A689A42A5
:10487C0009D8BB681A4607F1100319889B78118078
:10488C009370012300E0002318461837BD4680BD05
:10489C0080B592B000AFFCF731FD00F051FA00F09A
:1048AC009BFB00F073FB00F0F3FA00F01BFB00F035
:1048BC0043FB00F0A3FAFFF71BFFFFF765FBFFF7C5
:1048CC00E9FE1922A749A848FEF767FBA64B1B680F
:1048DC00DA68A54B1B6842F01002DA601922A34972
:1048EC00A348FEF75AFBA24B1B68DA68A04B1B6867
:1048FC0042F01002DA609F499F48FFF743FF9F4B3D
:10490C009B78FF2B0BD09D4BDB78FF2B07D09B4B61
:10491C009B78002B03D0994BDB78002B7FD14FF485
:10492C007A60FCF71DFD964801F0B2FA954801F04B
:10493C00AFFAFFF7D9FA4FF4FA60FCF711FD924881
:10494C0001F0A6FAFFF7E0FA4FF4FA60FCF708FD65
:10495C008E4801F09DFAFFF707FB4FF4FA60FCF765
:10496C00FFFC8B4801F094FAFFF7DEFA4FF4FA6083
:10497C00FCF7F6FC874801F08BFA0320FFF710FBDD
:10498C004FF4FA60FCF7ECFC834B7B64786CFBF720
:10499C00D7FB03469AB24FF0FF33796C7448FEF79D
:1049AC0071FA4FF4FA60FCF7DBFC7C4B3B64386C1F
:1049BC00FBF7C6FB03469AB24FF0FF33396C6C48D9
:1049CC00FEF760FA4FF4FA60FCF7CAFC744BFB6319
:1049DC00F86BFBF7B5FB03469AB24FF0FF33F96B5C
:1049EC006348FEF74FFA4FF4FA60FCF7B9FC634BDF
:1049FC009B78FF2B17D1614BDB78FF2B13D1F86B16
:104A0C00FBF79EFB03469AB24FF0FF33F96B584805
:104A1C00FEF738FA4FF47A60FCF7A2FCE7E761483E
:104A2C0001F036FA00E000BFFCF790FC0346184694
:104A3C0001F052F8514B9B781946504BDB781A46D3
:104A4C00594801F0BDF94D4B1B7A1946574801F0F6
:104A5C00B7F94A4B1B781946554801F0B1F9474B49
:104A6C001B78002B09D10A2252495348FFF7E2FE6A
:104A7C000346002B01D0FFF7EBFA404B1B7A03F0F7
:104A8C000F03002B05D03D4B1B7A03F0F003002BDA
:104A9C0005D1002249494848FBF7C2FE0BE04FF410
:104AAC00966246494448FFF7C5FE0346002B02D0E8
:104ABC00324B00221A72314B1B7A03F00F03002B7E
:104ACC0007D12E4B1B7A03F0F003102B01D1FFF70B
:104ADC0039FC2A4B1B7A03F00F03032B40F0A08008
:104AEC00264B1B78002B00F09B80244B1B7A03F089
:104AFC00F003F02B00F08380F02B00F38780202B49
:104B0C0002D0302B07D081E01C4B0222DA711B4BF8
:104B1C0033221A7284E007F1200300221A605A60D3
:104B2C009A60DA601A615A611A7607F12003194605
:104B3C002348FFF75FFD0346002B43D10F4B9A7CB4
:104B4C000E4BDB7C9A423DD207F120030021184624
:104B5C00FFF7AEFA094B9B7C0133DAB2074B9A7420
:104B6C0047E000BF24050020540400205C05002011
:104B7C000C040020BB000020BA000020B80000206C
:104B8C00F472000808730008247300083C730008D2
:104B9C005473000868730008807300088C73000855
:104BAC0098730008A8730008B4730008D073000849
:104BBC00E8730008A4030020B0030020AC0300201D
:104BCC00CC0000203B1D00221A605A609A60DA600B
:104BDC001A615A611A763B1D01211846FFF768FAD3
:104BEC00524B0122DA71514BF3221A72504801F0E8
:104BFC004FF94E4B1B8A1846FCF7B2FB10E04B4B9F
:104C0C0000221A82494B00221A7209E0494B0022F9
:104C1C001A70464B00221A82444B00221A7200BFB3
:104C2C00424B1B7A03F00F03082B1DD13F4B1B7813
:104C3C00002B19D03D4B1B7A03F0F003202B02D034
:104C4C00F02B06D009E0FFF703FA384BF3221A7267
:104C5C000AE0364B00221A7206E0344B00221A721C
:104C6C00354801F015F900BF304B1B7A03F00F03E8
:104C7C00072B3CD12D4B1B78002B38D02B4B1B7AA0
:104C8C0003F0F003F02B25D0F02B29DC202B02D0E5
:104C9C00302B15D024E0254B5B781846FFF780F9B4
:104CAC004FF4FA60FCF75CFB204B5B78032B03D1D1
:104CBC001E4BF7221A721AE01C4B37221A7216E09E
:104CCC00FFF79CF94FF4FA60FCF74AFB174BF722FD
:104CDC001A720CE0FFF7BCF9144B00221A7206E0B2
:104CEC00164801F0D5F8114B00221A7200BF0F4B79
:104CFC001B7A03F00F03052B7FF4A5AE0B4B1B782F
:104D0C00002B3FF4A0AEFFF7EDFA4FF4FA60FCF77E
:104D1C0027FBFFF719F94FF4FA60FCF721FB034B63
:104D2C00DB681846FFF752FB8DE600BFB800002089
:104D3C000074000875050020107400083474000815
:104D4C0080B594B000AF07F1280328220021184643
:104D5C0001F0A0F907F1140300221A605A609A605E
:104D6C00DA601A613B1D00221A605A609A60DA60A0
:104D7C000523BB624FF48033FB6200233B630123AA
:104D8C007B630123BB6302237B644FF48033BB64DE
:104D9C004FF4E013FB6407F128031846FCF704FBFF
:104DAC000346002B01D000F0C1F90F237B610223D5
:104DBC00BB610023FB614FF480633B6200237B6289
:104DCC0007F1140302211846FCF770FD0346002B73
:104DDC0001D000F0ABF901237B604FF48073BB6012
:104DEC003B1D1846FCF720FF0346002B01D000F0BA
:104DFC009DF900BF5037BD4680BD000080B582B024
:104E0C0000AF3B1D00210A461A800A469A70002307
:104E1C003B601D4B1D4A1A601B4B4FF0FF325A6012
:104E2C00194B4FF480729A601748FBF7D5FB034679
:104E3C00002B01D000F07AF900233B7100237B7129
:104E4C000023BB713B1D002219460F48FBF750FC99
:104E5C000346002B01D000F069F901233B700123BC
:104E6C007B700123BB700023FB703B46002219466C
:104E7C000548FBF7ADFD0346002B01D000F056F9B9
:104E8C0000BF0837BD4680BDB0030020002800409D
:104E9C0080B500AF114B124A1A60104B4FF4E1323F
:104EAC005A600E4B00229A600C4B0022DA600B4BBE
:104EBC0000221A61094B0C225A61084B00229A619C
:104ECC00064B0022DA610548FDF78CFF0346002BE8
:104EDC0001D000F02BF900BF80BD00BFC40300203F
:104EEC000038014080B500AF114B124A1A60104BCC
:104EFC004FF4E1325A600E4B00229A600C4B0022A8
:104F0C00DA600B4B00221A61094B0C225A61084BD8
:104F1C0000229A61064B0022DA610548FDF762FF18
:104F2C000346002B01D000F001F900BF80BD00BF8B
:104F3C000C0400200044004080B500AF114B124A15
:104F4C001A60104B4FF4E1325A600E4B00229A60FB
:104F5C000C4B0022DA600B4B00221A61094B0C221D
:104F6C005A61084B00229A61064B0022DA6105480F
:104F7C00FDF738FF0346002B01D000F0D7F800BF37
:104F8C0080BD00BF540400200048004080B582B0B2
:104F9C0000AF104B5B690F4A43F0010353610D4B9B
:104FAC005B6903F001037B607B68002200210D200C
:104FBC00FDF7C9FC0D20FDF7E2FC002200211020BA
:104FCC00FDF7C1FC1020FDF7DAFC00BF0837BD4629
:104FDC0080BD00BF0010024080B588B000AF07F163
:104FEC00100300221A605A609A60DA60424B9B6987
:104FFC00414A43F0100393613F4B9B6903F010034C
:10500C00FB60FB683C4B9B693B4A43F0200393617C
:10501C00394B9B6903F02003BB60BB68364B9B6923
:10502C00354A43F004039361334B9B6903F004034B
:10503C007B607B68304B9B692F4A43F0080393617C
:10504C002D4B9B6903F008033B603B6801224FF436
:10505C0080712A48FDF7EFF800224FF400412748F1
:10506C00FDF7E9F8002208212548FDF7E4F84FF494
:10507C0040433B61234B7B610123BB6107F1100370
:10508C0019461F48FCF73CFF4FF480733B6101232A
:10509C007B610123BB610223FB6107F110031946FD
:1050AC001648FCF72DFF4FF400433B6101237B6155
:1050BC000223BB610223FB6107F1100319460F4861
:1050CC00FCF71EFF08233B6101237B610223BB61BC
:1050DC000223FB6107F1100319460948FCF710FF86
:1050EC00002200212820FDF72EFC2820FDF747FC8C
:1050FC0000BF2037BD4680BD0010024000080140B3
:10510C00000C01400000311080B582B000AF786017
:10511C007B681B68044A934201D1FCF705F900BF78
:10512C000837BD4680BD00BF0004004080B400AF0E
:10513C0072B600BF00BFFDE780B400AF00BFFDE753
:10514C0080B400AF00BFFDE780B400AF00BFFDE747
:10515C0080B400AF00BFFDE780B400AF00BFFDE737
:10516C0080B400AF00BFBD4680BC704780B400AFB8
:10517C0000BFBD4680BC704780B400AF00BFBD46C9
:10518C0080BC704780B400AF00BFBD4680BC704788
:10519C0080B500AF0248FDF7EDF900BF80BD00BF40
:1051AC00E004002080B500AF0248FDF7E3F900BF32
:1051BC0080BD00BF9C04002080B500AF0248FBF707
:1051CC0077F800BF80BD00BF7805002080B586B0A1
:1051DC0000AF6248FDF786FF604B1B681B6803F04D
:1051EC001003102B40F0B5800023BB605B4B1B6899
:1051FC001B68BB60594B1B685B68BB60BB6857483E
:10520C00FDF7F0FE554BDB6B1B685B689BB2C3F183
:10521C001903FB82FB8A002B00F09180FB8A092B7F
:10522C0041D94F4B1B78552B3DD14D4B5B78BB2B4C
:10523C0039D14B4BDA784B4B9B789A4233D1484B54
:10524C001A79484BDB789A422DD1454B9B7AFF2B30
:10525C0029D1434BDB7AEE2B25D1424B1B7A03F041
:10526C000F03002B14D13F4B1B7A03F0F003002BE0
:10527C000ED1FB8A1A463A493B4800F0C2FF394B23
:10528C0010221A7236493948FFF77AF900BF55E0F7
:10529C00334B9B780A2B51D1324B01221A70314B74
:1052AC0000221A724AE0FB8A062B07D907223049E2
:1052BC002B4800F0F7FE0346002B40D0FB8A012B55
:1052CC003DD902222B49264800F0ECFE0346002B68
:1052DC0035D12949224800F00AFF38613B69002B7F
:1052EC002DD03B690B333B613B691D4A9B1ADA1C81
:1052FC00FB8A9A4223DA3B4600221A601A713B461B
:10530C0004223969184600F0DFFE3B4610220021CA
:10531C00184600F089FCF860FB681B12DAB2114BDE
:10532C009A70FB68DAB20F4BDA700E4B9B780D4A11
:10533C00D27811461846FFF7EFF900E000BF1922AA
:10534C000021074800F0A6FE192205490348FDF785
:10535C0024FE00BF1837BD4680BD00BF0C040020E2
:10536C005C050020B8000020400500203802002019
:10537C0048740008507400085474000880B584B058
:10538C0000AF2048FDF7AEFE1E4B1B681B6803F0F8
:10539C001003102B32D10023FB601A4B1B681B68C7
:1053AC00FB60184B1B685B68FB60FB681548FDF7DE
:1053BC0019FE02221449154800F074FE0346002B16
:1053CC0012D0134BDB79012B0ED11248FFF7B2F838
:1053DC000346002B04D03B4619460E48FFF70AF94A
:1053EC000A490C48FFF7CCF819220021074800F0B5
:1053FC0051FE192205490348FDF7CFFD00BF1037B8
:10540C00BD4680BD540400205074000824050020C3
:10541C00B8000020CC00002080B500AF4FF48040D5
:10542C00FCF722FF4FF40040FCF71EFF00BF80BDCD
:10543C0080B500AF0348FBF78DFC034800F028FD56
:10544C0000BF80BDB00300206074000880B584B03C
:10545C0000AF0346FB8007F10C0300210A461A80BB
:10546C000A469A7007F10C03002219461D48FBF7F7
:10547C00D7F9FB88B3F5804F17D14FF480411A4808
:10548C00FCF7C2FE0346012B03D1184800F000FDC7
:10549C0024E0174800F0FCFC164B1A4607F10C03ED
:1054AC0019889B781180937018E0FB88B3F5004F36
:1054BC0014D14FF400410C48FCF7A6FE0346012B17
:1054CC0003D10D4800F0E4FC08E00C4800F0E0FCCF
:1054DC0000224FF480710A48FCF7ADFE00BF103774
:1054EC00BD4680BDB0030020000C01407074000864
:1054FC0080740008A803002090740008A4740008AD
:10550C000008014080B485B000AF154B9B69144A6C
:10551C0043F001039361124B9B6903F00103BB60E1
:10552C00BB680F4BDB690E4A43F08053D3610C4BC5
:10553C00DB6903F080537B607B680A4B5B68FB6024
:10554C00FB6823F0E063FB60FB6843F00073FB60D7
:10555C00044AFB68536000BF1437BD4680BC7047DB
:10556C00001002400000014080B584B000AF7860AC
:10557C007B681B680F4A934218D1FDF70FFA0E4B4C
:10558C00DB690D4A43F00063D3610B4BDB6903F01D
:10559C000063FB60FB68094B01221A6000220021AA
:1055AC002920FDF7D0F92920FDF7E9F900BF1037C4
:1055BC00BD4680BD00280040001002403C04424221
:1055CC0080B58CB000AF786007F1200300221A6020
:1055DC005A609A60DA607B681B68824A934232D1C7
:1055EC00814B9B69804A43F4804393617E4B9B695A
:1055FC0003F48043FB61FB697B4B9B697A4A43F064
:10560C0004039361784B9B6903F00403BB61BB6992
:10561C004FF400733B6202237B620323FB6207F1AE
:10562C00200319467148FCF76BFC4FF480633B6216
:10563C0000237B620023BB6207F1200319466B48F1
:10564C00FCF75EFCCAE07B681B68694A93425FD139
:10565C00654BDB69644A43F40033D361624BDB690D
:10566C0003F400337B617B695F4B9B695E4A43F0BB
:10567C00040393615C4B9B6903F004033B613B693E
:10568C0004233B6202237B620323FB6207F12003AA
:10569C0019465648FCF734FC08233B6200237B6216
:1056AC000023BB6207F1200319465048FCF728FC85
:1056BC00504B514A1A604F4B00225A604D4B0022FE
:1056CC009A604C4B8022DA604A4B00221A61494B9B
:1056DC0000225A61474B00229A61464B4FF400520C
:1056EC00DA614448FCF7D8FD0346002B01D0FFF7E4
:1056FC001DFD7B683F4ADA633E4A7B685362002299
:10570C0000212620FDF71FF92620FDF738F965E06A
:10571C007B681B68394A934260D1334BDB69324A50
:10572C0043F48023D361304BDB6903F48023FB60AB
:10573C00FB682D4B9B692C4A43F0080393612A4B61
:10574C009B6903F00803BB60BB684FF480633B624A
:10575C0002237B620323FB6207F1200319462848CE
:10576C00FCF7CEFB4FF400633B6200237B6200230B
:10577C00BB6207F1200319462148FCF7C1FB214B02
:10578C00214A1A601F4B00225A601E4B00229A605D
:10579C001C4B8022DA601B4B00221A61194B002231
:1057AC005A61184B00229A61164B4FF40052DA6181
:1057BC001448FCF771FD0346002B01D0FFF7B6FC33
:1057CC007B68104ADA630F4A7B685362002200211F
:1057DC002720FDF7B8F82720FDF7D1F800BF3037A8
:1057EC00BD4680BD00380140001002400008014059
:1057FC00004400409C0400206C0002400048004023
:10580C00000C0140E00400203000024080B58EB056
:10581C0000AF78600023FB620023BB62002387F893
:10582C003330344BDB69334A43F00203D361314BE1
:10583C00DB6903F00203FB60FB6807F1100207F160
:10584C00140311461846FCF7A1F93B6AFB62FB6A8C
:10585C00002B03D1FCF772F9786304E0FCF76EF9C6
:10586C0003465B007B637B6B234AA2FB03239B0CED
:10587C00013BBB62214B224A1A60204B40F2E732BB
:10588C00DA601E4ABB6A53601C4B00221A611B4B28
:10589C0000229A60194B00229A611848FAF75EFCB4
:1058AC00034687F8333097F83330002B1BD113485D
:1058BC00FAF7ACFC034687F8333097F83330002BFB
:1058CC0011D11D20FDF75BF87B680F2B08D8002247
:1058DC0079681D20FDF737F80A4A7B68136002E0EF
:1058EC00012387F8333097F8333018463837BD46E4
:1058FC0080BD00BF0010024083DE1B4378050020F2
:10590C00000400400400002080B586B000AF786031
:10591C00144A154BD31A7B617B693B61134B1B6893
:10592C00002B02D1114B124A1A60104B1A687B687B
:10593C0013443A699A4207D200F036FC03460C2213
:10594C001A604FF0FF3309E0084B1B68FB60074BF4
:10595C001A687B681344054A1360FB6818461837AD
:10596C00BD4680BD0050002000040000C005002092
:10597C001007002080B400AF01231846BD4680BC40
:10598C00704780B582B000AF7860396000F00CFCD5
:10599C00034616221A604FF0FF3318460837BD46EF
:1059AC0080BD80B582B000AF78604FF0FF31786871
:1059BC00FFF7E7FF00BFFDE780B586B000AFF860EA
:1059CC00B9607A6000237B610AE0AFF30080014686
:1059DC00BB685A1CBA60CAB21A707B6901337B610E
:1059EC007A697B689A42F0DB7B6818461837BD46AB
:1059FC0080BD80B586B000AFF860B9607A600023D6
:105A0C007B6109E0BB685A1CBA601B781846FEF72C
:105A1C002BFE7B6901337B617A697B689A42F1DBEF
:105A2C007B6818461837BD4680BD80B483B000AF84
:105A3C0078604FF0FF3318460C37BD4680BC70477A
:105A4C0080B483B000AF786039603B684FF400528B
:105A5C005A60002318460C37BD4680BC704780B492
:105A6C0083B000AF7860012318460C37BD4680BC6C
:105A7C00704780B485B000AFF860B9607A600023DD
:105A8C0018461437BD4680BC70470000FAF760FB1F
:105A9C000B480C490C4A002302E0D458C450043380
:105AAC00C4188C42F9D3094A094C002301E0136055
:105ABC000432A242FBD300F07DFBFEF7E9FE7047F7
:105ACC000000002078000020E87600087800002014
:105ADC0010070020FEE7000038B5104B04461D6887
:105AEC002B6BB3B9182000F001FC0246286320B9D7
:105AFC0046210B4B0B4800F093FB0B490B4BC0E9B9
:105B0C0000130B4B002183600B2383810120C2E91E
:105B1C00040100222B6B1C615A6138BD2800002047
:105B2C00F67400080D7500080E33CDAB34126DE61B
:105B3C00ECDE0500242B2DE9F0478646904601D873
:105B4C00012B06D100F030FB162303600020BDE8CA
:105B5C00F0870D4633482A4615F8014B065D16F0C2
:105B6C000806F8D12D2C10D101262C78951C33F079
:105B7C00100215D1302C0DD12A7802F0DF02582AF0
:105B8C0008D16C78023510230AE02B2C04BF2C783A
:105B9C00951CECE7002BF6D1302C14BF0A230823FC
:105BAC00002206F1004C0CF1FF3CBCFBF3F9104653
:105BBC0003FB19CAA4F13007092F0FD83C46A342A6
:105BCC001BDD571C07D0814514D301D1A24511DB35
:105BDC00012200FB034015F8014BEBE7A4F1410750
:105BEC00192F01D8373CEAE7A4F16107192F04D823
:105BFC00573CE4E74FF0FF32EDE7531C08D122236A
:105C0C006046CEF80030B8F1000FA0D0691E06E057
:105C1C0006B14042B8F1000F99D0002AF6D1C8F86D
:105C2C00001094E7D575000813460A460146024851
:105C3C000068FFF77FBF00BF28000020002310B5CD
:105C4C000446C0E90033C0E90433836081814366B4
:105C5C00C2818361194608225C3000F01BFA0D4B9F
:105C6C00246263620C4BA3620C4BE3620C4B236308
:105C7C000C4B9C4206D003F16802944202D0D03304
:105C8C009C4205D104F15800BDE8104000F0B6BAB2
:105C9C0010BD00BFF15E0008135F00084B5F0008E9
:105CAC006F5F0008C4050020024A0349034800F056
:105CBC0069B800BF1C000020B56D00082C00002046
:105CCC0041680C4B10B59942044601D001F06CF8B8
:105CDC00A168094B994202D0204601F065F8E168B1
:105CEC00064B994204D02046BDE8104001F05CB848
:105CFC0010BD00BFC40500202C0600209406002017
:105D0C0010B50B4B0B4C0C4A20461A600421002298
:105D1C00FFF794FF04F1680001220921FFF78EFFC1
:105D2C0004F1D0000222BDE810401221FFF786BF1B
:105D3C00FC060020C4050020B55C0008014800F0FA
:105D4C005EBA00BF05070020014800F059BA00BF39
:105D5C000507002010B50446FFF7F0FF236A1BB1BE
:105D6C00BDE81040FFF7F0BF044B2362044B1B68E7
:105D7C00002BF5D1FFF7C4FFF2E700BFCD5C0008A4
:105D8C00FC0600202DE9F8430746884614460026F9
:105D9C00D4E90195B9F1010905D52468002CF7D196
:105DAC003046BDE8F883AB89012B07D9B5F90E3025
:105DBC00013303D029463846C04706436835E9E726
:105DCC000FB407B5064904AB086853F8042B816877
:105DDC00019300F0C1FC03B05DF804EB04B0704714
:105DEC0028000020036A70B505460E4684680BB97E
:105DFC00FFF7B0FF636EDB0705D4A389980502D4C7
:105E0C00A06D00F0FCF9A389190702D52369002BBA
:105E1C0035D12146284600F0E7F880B34FF0FF3526
:105E2C00636EDA0705D4A3899B0502D4A06D00F03C
:105E3C00E7F9284670BD002B04DAA2699A4217DCF8
:105E4C000A2915D023685A1C22601970A36816F809
:105E5C00011F013BA3600029EDD1002B11DA224672
:105E6C000A21284600F081F80130D7D00A25D7E75F
:105E7C002246284600F079F80130E7D1CEE7013E02
:105E8C00E4E723685A1C22600A221A70EEE700002D
:105E9C00024B01461868FFF7A5BF00BF2800002081
:105EAC000EB46FF0004110B500249DB01FAB0290F2
:105EBC000690079104910948094953F8042B059160
:105ECC00006802A901931B9400F022FB029B1C703A
:105EDC001DB0BDE8104003B0704700BF2800002083
:105EEC000802FFFF10B50C46B1F90E1000F038F99E
:105EFC000028ABBF636DA3891B1823F48053ACBF80
:105F0C006365A38110BD2DE9F0411F468B890546C1
:105F1C00DB050C46164605D502230022B1F90E10FE
:105F2C0000F00CF9A389324623F48053A381284650
:105F3C003B46B4F90E10BDE8F04100F023B910B5A2
:105F4C000C46B1F90E1000F0F9F8431CA38915BFEB
:105F5C00606523F4805343F48053A38118BFA3815D
:105F6C0010BDB1F90E1000F0D9B8F8B50E461446B4
:105F7C00054618B1036A0BB9FFF7ECFEA369A360E1
:105F8C00A3891A0701D5236943B92146284600F095
:105F9C002BF818B14FF0FF373846F8BD236822694B
:105FAC00F6B2981A63693746834205DC21462846C7
:105FBC0000F0FAFE0028EDD1A368013BA360236832
:105FCC005A1C22601E706269431C9A4204D0A38939
:105FDC00DB07E1D50A2EDFD12146284600F0E4FE8E
:105FEC000028D9D0D6E7000038B5294B05461868EB
:105FFC000C4618B1036A0BB9FFF7ACFEB4F90C30C0
:10600C00190722D4DA0607D409222A6043F0400388
:10601C004FF0FF30A38133E0580712D5616B41B1CB
:10602C0004F14403994202D0284600F017F90023EA
:10603C006363A38923F02403A38100236360236992
:10604C002360A38943F00803A38123694BB9A38977
:10605C0003F42073B3F5007F03D02146284600F0EB
:10606C0002FFB4F90C3013F001020AD00022A26036
:10607C0062695242A261226942B913F08000C5D113
:10608C0038BD990758BF6269A260F4E70020F7E7B2
:10609C002800002003460244934200D1704703F8C5
:1060AC00011BF9E710B56AB10139841810F8012BFE
:1060BC0011F8013F9A4203D1A04201D0002AF5D138
:1060CC00D01A10BD1046FCE7034610B5013932B1A9
:1060DC0011F8014F013A03F8014B002CF7D10021C4
:1060EC001A44934200D110BD03F8011BF9E70A785A
:1060FC0070B56AB970BD9A4209D10C46054614F8C0
:10610C00013F002BF6D015F8016F9E42F7D00130FD
:10611C000378002BEFD11846ECE7000038B50023CC
:10612C00054D044608462B60FFF77FFC431C02D14B
:10613C002B6803B1236038BD0007002038B5044636
:10614C00084611460022054D2A601A46FFF791FCBD
:10615C00431C02D12B6803B1236038BD000700201B
:10616C0038B50446084611460022054D2A601A46E9
:10617C00FFF722FC431C02D12B6803B1236038BD0E
:10618C000007002038B50446084611460022054D8C
:10619C002A601A46FFF72DFC431C02D12B6803B171
:1061AC00236038BD00070020014B1868704700BF02
:1061BC002800002070B500260C4D0D4C641BA4105B
:1061CC00A64209D100F068FF00260A4D0A4C641B58
:1061DC00A410A64205D170BD55F8043B9847013672
:1061EC00EEE755F8043B98470136F2E7E0760008F5
:1061FC00E0760008E0760008E47600087047704707
:10620C0070470A44914200F1FF3300D1704710B53A
:10621C0011F8014B914203F8014FF9D110BD000068
:10622C001FB514461A46094B05461B68D8684CB175
:10623C00074BCDE9013400912B46064900F0DCFDFB
:10624C0000F0A8FE044B1C46F3E700BF280000201A
:10625C006575000872750008A075000838B505460C
:10626C00002940D051F8043C0C1F002BB8BFE41897
:10627C0000F0E6F81C4A136833B9636014602846D2
:10628C00BDE8384000F0E2B8A34208D920682118D4
:10629C008B4201BF19685B6809182160EDE71A464B
:1062AC005B680BB1A342FAD911685018A0420BD10C
:1062BC0020680144501883421160E0D118685B6873
:1062CC00084410605360DAE702D90C232B60D6E740
:1062DC00206821188B4201BF19685B68091821607E
:1062EC0063605460CBE738BD0C070020024B0146BD
:1062FC00186800F025B800BF2800002070B50F4EBC
:10630C000C463168054611B900F026FE3060214676
:10631C00284600F021FE431C03D14FF0FF342046E9
:10632C0070BDC41C24F00304A042F8D0211A2846E6
:10633C0000F012FE0130F2D1EFE700BF0807002099
:10634C002DE9F843CD1C25F0030508350C2D38BF7D
:10635C000C25002D064601DBA94204D90C23336021
:10636C000020BDE8F883DFF8D48000F069F8D8F895
:10637C0000301C4644BB29463046FFF7BFFF431C88
:10638C00044658D1D8F800402746002F43D1002CA2
:10639C004BD023683946304604EB030900F0DCFD92
:1063AC00814542D1216830466D1A2946FFF7A6FF78
:1063BC0001303AD023682B442360D8F800305A6857
:1063CC0062BBC8F800700FE02268521B20D40B2A65
:1063DC0017D96119A342256018BF5960636808BFBB
:1063EC00C8F8001062514B60304600F02FF804F1F1
:1063FC000B00231D20F00700C21A1CBF1B1AA35050
:10640C00AFE76268A3420CBFC8F800205A60EBE704
:10641C0023466468AEE73C467F68B6E71A465B687D
:10642C00A342FBD100235360DEE70C2330463360DC
:10643C0000F00CF894E70560D6E700BF0C070020CD
:10644C000148FFF7DCBE00BF040700200148FFF73E
:10645C00D7BE00BF040700202DE9F0471F468E6809
:10646C008246BE420C4690460B682DD8B1F90C20E2
:10647C0012F4906F26D06569096905EB4505A3EB0D
:10648C00010905EBD5757B1C4B446D109D4238BF43
:10649C001D46530527D52946FFF752FF064660B324
:1064AC004A462169FFF7ADFEA38923F4906343F0BC
:1064BC008003A38126614E4426603E466561A5EBB0
:1064CC000905A560BE4200D93E46324641462068C9
:1064DC0000F005FD0020A3689B1BA36023683344D8
:1064EC002360BDE8F0872A4600F05BFD06460028D5
:1064FC00E0D150462169FFF7B1FE0C23CAF80030F9
:10650C00A3894FF0FF3043F04003A381E9E700007B
:10651C002DE9F04F98468B8907461B060D4614460D
:10652C009DB010D50B6973B94021FFF709FF2860A6
:10653C00286130B90C233B604FF0FF301DB0BDE833
:10654C00F08F40236B610023099320238DF82930B1
:10655C0030234FF00109CDF80C80DFF898818DF8CD
:10656C002A3023469A4613F8012B0AB1252AF9D171
:10657C00BAEB040B0BD05B46224629463846FFF794
:10658C006BFF013000F0A780099A5A4409929AF8DF
:10659C000030002B00F09F8000234FF0FF32CDE93C
:1065AC0005230AF1010A049307938DF853301A93CB
:1065BC005446052214F8011B4E4800F0DDFC049AE9
:1065CC00D8B9D00644BF20238DF85330110744BFEF
:1065DC002B238DF853309AF800302A2B15D05446C3
:1065EC0000204FF00A0C079A214611F8013B303B72
:1065FC00092B4BD9B0B1079214E0A0EB080309FAB0
:10660C0003F31343A2460493D2E7039B191D1B68A3
:10661C000391002BBBBF5B4242F00202079307932E
:10662C00B8BF049223782E2B0AD163782A2B32D14F
:10663C00039B02341A1D1B68039243EAE373059310
:10664C00DFF8B4A003225046217800F095FC38B155
:10665C004022049BA0EB0A008240134301340493B4
:10666C0014F8011B062225488DF8281000F084FC34
:10667C00002836D0224B1BBB039B073323F00703A8
:10668C0008330393099B334409936AE70C460120B2
:10669C000CFB0232A8E700234FF00A0C1946013418
:1066AC000593204610F8012B303A092A03D9002B08
:1066BC00C6D00591C4E7044601230CFB0121F0E789
:1066CC0003AB00932A4638460E4B04A9AFF3008067
:1066DC00421C0646D6D1AB895B063FF52DAF099817
:1066EC002CE703AB00932A463846064B04A900F06E
:1066FC00BDF9EDE7A1750008A7750008AB7500089A
:10670C000000000065640008936810B4013B002B86
:10671C00936007DA9469A34201DB0A2902D110BC09
:10672C00FFF723BC1368581C10601970084610BC86
:10673C007047F8B506460F461446D518AC4201D141
:10674C00002007E03A46304614F8011BFFF7DCFF47
:10675C00431CF3D1F8BD00002DE9F04F0D46144653
:10676C00984606469DB018B1036A0BB9FFF7F2FACA
:10677C006B6ED90705D4AB899A0502D4A86DFFF7C7
:10678C003EFDAB891B0701D52B699BB929463046C9
:10679C00FFF72AFC70B16B6EDC0704D54FF0FF30AD
:1067AC001DB0BDE8F08FAB899805F7D4A86DFFF745
:1067BC0027FDF3E70023099320238DF8293030239C
:1067CC004FF00109CDF80C80DFF8A8818DF82A3044
:1067DC0023469A4613F8012B0AB1252AF9D1BAEBB4
:1067EC00040B0BD05B46224629463046FFF7A1FF2F
:1067FC00013000F0A780099A5A4409929AF80030A7
:10680C00002B00F09F8000234FF0FF32CDE90523D1
:10681C000AF1010A049307938DF853301A935446E6
:10682C00052214F8011B534800F0A6FB049AD8B9B2
:10683C00D10644BF20238DF85330130744BF2B23BC
:10684C008DF853309AF800302A2B15D0544600207E
:10685C004FF00A0C079A214611F8013B303B092BEB
:10686C004BD9B0B1079214E0A0EB080309FA03F37B
:10687C001343A2460493D2E7039B191D1B68039193
:10688C00002BBBBF5B4242F0020207930793B8BFD9
:10689C00049223782E2B0AD163782A2B32D1039BB6
:1068AC0002341A1D1B68039243EAE3730593DFF865
:1068BC00C8A003225046217800F05EFB38B140227C
:1068CC00049BA0EB0A00824013430134049314F898
:1068DC00011B062229488DF8281000F04DFB0028DA
:1068EC003FD0274B1BBB039B073323F00703083315
:1068FC000393099B3B4409936AE70C4601200CFB6C
:10690C000232A8E700234FF00A0C19460134059314
:10691C00204610F8012B303A092A03D9002BC6D097
:10692C000591C4E7044601230CFB0121F0E703ABFE
:10693C0000932A463046134B04A9AFF30080074658
:10694C00781CD6D16B6ED90705D4AB899A0502D4C5
:10695C00A86DFFF755FCAB895B063FF51FAF099897
:10696C001EE703AB00932A463046064B04A900F001
:10697C007DF8E4E7A1750008A7750008AB75000861
:10698C00000000003F6700082DE9F04716469846C6
:10699C008A680B6907469342B8BF1346336091F877
:1069AC0043200C46DDF820900AB101333360236894
:1069BC00990642BF336802333360256815F006052B
:1069CC0006D104F1190AE36832689B1AAB422BDC3E
:1069DC0094F843302268003B18BF0123920630D450
:1069EC004146384604F14302C847013023D023689E
:1069FC00226903F00603042B14BF002533684FF003
:106A0C00000608BFE56804F11A0408BFED1A54F833
:106A1C00123C08BF25EAE5759342C4BF9B1AED18DA
:106A2C00B5421AD1002008E00123524641463846AF
:106A3C00C847013003D14FF0FF30BDE8F087013576
:106A4C00C1E73020E11881F843005A1C94F8451036
:106A5C002244023382F84310C2E701232246414606
:106A6C003846C8470130E6D00136D9E72DE9FF4753
:106A7C000F7E9146782F80460C469A460C9E01F16B
:106A8C00430207D8622F0AD8002F00F0D180582F6C
:106A9C0000F0B88004F1420684F842703AE0A7F1A5
:106AAC006303152BF6D801A151F823F0116B0008E4
:106ABC00256B0008A16A0008A16A0008A16A0008F9
:106ACC00A16A0008256B0008A16A0008A16A0008E9
:106ADC00A16A0008A16A0008236C00084F6B00082B
:106AEC00DD6B0008A16A0008A16A0008456C00086B
:106AFC00A16A00084F6B0008A16A0008A16A00088F
:106B0C00E56B000833681A1D1B68326004F14206FD
:106B1C0084F8423001239CE033682068191D3160F1
:106B2C00060601D51D6803E04506FBD5B3F90050F8
:106B3C00002D03DA2D236D4284F843300A23584884
:106B4C0011E021683368080653F8045B02D4490647
:106B5C0048BFADB26F2F336014BF0A2308235048CF
:106B6C00002184F843106668002EA66005DB2168BE
:106B7C002E4321F0040121604BD01646B5FBF3F1F6
:106B8C0003FB1157C75D06F8017D2F46BB420D462E
:106B9C00F4D9082B0BD12368DF0708D5236961686A
:106BAC009942DEBF302306F8013C06F1FF36921BFA
:106BBC0022614B4621464046CDF800A003AAFFF7C0
:106BCC00E3FE01304AD14FF0FF3004B0BDE8F0874E
:106BDC00236843F0200323607827324884F84570FB
:106BEC00236831681F0651F8045B02D45F0648BF66
:106BFC00ADB23160D90744BF43F0200323601DB10F
:106C0C001023ADE72648E9E7236823F0200323602F
:106C1C00F6E71646BDE733682568181D61693060D4
:106C2C002E061B6801D5196002E06806FBD5198099
:106C3C00002316462361BCE7336800211A1D32601D
:106C4C001E686268304600F097F908B1801B6060DE
:106C5C0063682361002384F84330AAE7324649462F
:106C6C0040462369D0470130ADD023689B0713D42D
:106C7C00E068039B9842B8BF1846A6E7012332464A
:106C8C0049464046D04701309DD00135E368039911
:106C9C005B1AAB42F2DCEBE7002504F11906F5E7D1
:106CAC00B2750008C3750008B1F90C20F8B51607C9
:106CBC0005460C4654D44B68002B02DC0B6C002BA5
:106CCC0048DDE66A002E45D0002312F480522F686E
:106CDC00216A2B6030D0626DA389590705D5636892
:106CEC00D21A636B0BB1236CD21A00232846E66AC6
:106CFC00216AB047431CA38906D129681D292BD8CA
:106D0C00284ACA40D60727D5002262602269D904D6
:106D1C00226004D5421C01D12B6803B96065616BFC
:106D2C002F60B9B104F14403994202D02846FFF711
:106D3C0095FA002363630DE001232846B047024611
:106D4C00501CC9D12B68002BC6D01D2B01D0162B83
:106D5C001DD12F60002021E043F040031BB21AE04C
:106D6C000F69002FF6D0930718BF00230E6808BFD9
:106D7C004B69F61B0F608B60002EEBDD33463A46F9
:106D8C002846216AD4F828C0E047002807DCB4F96B
:106D9C000C3043F040034FF0FF30A381F8BD0744A3
:106DAC00361AE9E70100402038B50B6905460C4658
:106DBC0013B90025284638BD18B1036A0BB9FEF784
:106DCC00C9FFB4F90C30002BF3D0626ED00704D499
:106DDC00990502D4A06DFFF712FA28462146FFF759
:106DEC0063FF636E0546DA07E4D4A3899B05E1D4FF
:106DFC00A06DFFF705FADDE70EB403B5014603AB52
:106E0C00054853F8042B00680193FFF7A5FC02B06A
:106E1C005DF804EB03B070472800002070B50C46F9
:106E2C00B1F90E10154600291E4696B00CDAA3894E
:106E3C00002113F0800F14BF40234FF48063002017
:106E4C0031602B6016B070BD6A4600F063F8002804
:106E5C00EDDB019901F47041A1F500535942594100
:106E6C004FF48063EBE78B89F7B59D0706460C461C
:106E7C0007D504F14703236023610123636103B049
:106E8C00F0BD6A4601ABFFF7C9FF009F05463946C6
:106E9C003046FFF755FA48B9B4F90C309A05EED4E0
:106EAC0023F0030343F00203A381E2E7A389C4E9BF
:106EBC00040743F08003A381019B20605BB1304643
:106ECC00B4F90E1000F038F828B1A38923F00303AD
:106EDC0043F00103A381A3891D43A581CFE7884219
:106EEC0010B501EB020402D98442234607D8431E95
:106EFC00A14208D011F8012B03F8012FF8E7014645
:106F0C0002448A4200D110BD13F8014D02F8014D24
:106F1C00F7E7000038B50023064D04460846114635
:106F2C002B60FEF78DFD431C02D12B6803B123604F
:106F3C0038BD00BF0007002038B50023054D0446BE
:106F4C0008462B60FEF78BFD431C02D12B6803B166
:106F5C00236038BD0007002038B50023054D0446DA
:106F6C0008462B60FEF7D0FC431C02D12B6803B102
:106F7C00236038BD00070020034610B5C9B2024497
:106F8C009342184601D1002003E0047801338C426F
:106F9C00F6D110BD062008B500F05AF80120FEF716
:106FAC0000FD2DE9F041074614460D4621B9114666
:106FBC00BDE8F041FFF7C4B92AB9FFF74FF92546F0
:106FCC002846BDE8F08100F05FF88442064602D8FE
:106FDC00B4EB500FF4D821463846FFF7B1F9804690
:106FEC0008B94546ECE7B4422246294628BF32464A
:106FFC00FFF707F929463846FFF730F9F1E71F2963
:10700C0038B505460C4604D9162303604FF0FF3003
:10701C0038BDC26B12B152F821304BB9284600F082
:10702C0031F8224601462846BDE8384000F018B831
:10703C00012B0AD0591C03D1162303600120E7E76A
:10704C000021204642F8241098470020E0E7000079
:10705C00024B01461868FFF7D2BF00BF2800002082
:10706C0038B50023064D0446084611462B60FEF742
:10707C0088FC431C02D12B6803B1236038BD00BFD0
:10708C0000070020FEF776BC51F8043C181F002BBB
:10709C00BCBF0B58C0187047F8B500BFF8BC08BC93
:1070AC009E467047F8B500BFF8BC08BC9E467047BA
:1070BC0041542B524F4C453D3200000041542B5350
:1070CC0043414E494E54563D3530300041542B52BD
:1070DC00455345540000000041542B534C4545503A
:1070EC00000000004154000041542B5343414E57C3
:1070FC004E443D313238000041542B4453545F41CF
:10710C004444523D25752C3000000000E8BF99E640
:10711C0098AFE5BF83E8B7B3E58C850D00000000A0
:10712C00E8BF99E698AFE58F91E98081E8939DE7F8
:10713C008999E695B0E68DAE0D000000E8BF99E6A2
:10714C0098AFE58F91E98081534F53E695B0E68D6A
:10715C00AE0D0000E8BF99E698AFE8AFB7E6B18294
:10716C00E8939DE78999E695B0E68DAEE79A84E5BC
:10717C0091BDE4BBA40D0000E689ABE68F8FE697CA
:10718C00B6E997B4E4B8BA302CE9BB98E8AEA435AC
:10719C0030306D73E689ABE68F8FE697B6E997B41E
:1071AC000D000000E8BF99E698AFE9858DE7BDAE0C
:1071BC006C6F7261E58F91E98081E696B9E5BC8FC1
:1071CC00E79A84E591BDE4BBA40D0000E697A0E628
:1071DC009588E79A84E5B9BFE692ADE7B1BBE59E29
:1071EC008BEFBC8CE8AFB7E9878DE696B0E8BE9321
:1071FC00E585A50D00000000E8BF99E698AFE8AE64
:10720C00A9E8AEBEE5A487E79DA1E79CA0E79A8418
:10721C00E591BDE4BBA40D00E79DA1E79CA0E6971A
:10722C00B6E997B4E697A0E695882C20E4BDBFE7B5
:10723C0094A8E9BB98E8AEA4333030306D730D00E0
:10724C00E68EA5E694B6E588B0E79DA1E79CA0E69E
:10725C0097B6E997B43A20256C7520E7A7920D0AEA
:10726C0000000000E8BF99E698AFE8AEA9E8AEBE12
:10727C00E5A487E9878DE696B0E58F91E98081E7F3
:10728C0082B9E58DAFE591BDE4BBA40D0000000013
:10729C0041542B4F5054494F4E3D312C300000007F
:1072AC0041542B4F5054494F4E3D322C300000006E
:1072BC0041542B4F5054494F4E3D332C300000005D
:1072CC004572726F723A2064656C61795F736563A5
:1072DC006F6E6473206D7573742062652031207E2F
:1072EC002038363339390D00E5BC80E5A78BE588AD
:1072FC009DE5A78BE58C960D00000000E58887E6E0
:10730C008DA2E4B8BAE8A782E5AF9FE88085E6A82D
:10731C00A1E5BC8F0D000000E5889DE5A78BE58CF1
:10732C0096E689ABE68F8FE997B4E99A940D000045
:10733C00E5889DE5A78BE58C96E689ABE68F8FE714
:10734C00AA97E58FA30D0000E5889DE5A78BE58C3A
:10735C0096E5A48DE4BD8D0D00000000E5BC80E534
:10736C0090AF4C6F7261E5B9BFE692ADE6A8A1E5AE
:10737C009D970D0041542B545950453D3100000050
:10738C0041542B484541443D3000000041542B539F
:10739C0052435F414444523D3F000000E5B7B2E91F
:1073AC00858DE7BDAE0D0000E8AEBEE5A487E59C7B
:1073BC00B0E59D80EFBC9A307825303258253032BC
:1073CC00580A0000E8AEBEE5A487E78AB6E68081DD
:1073DC00EFBC9A3078253032580A00004465766943
:1073EC0063652069732072656164793A2025640DA8
:1073FC000A000000E58F91E98081E5AE8CE688906B
:10740C000D000000E694B6E588B0E69CAAE79FA5BF
:10741C00E6ADA5E9AAA4EFBC8CE5BFBDE795A5E553
:10742C00A484E790860D0000E69CAAE79FA5E98559
:10743C008DE7BDAEE591BDE4BBA40D0053554343B0
:10744C0045535300415400005352435F414444524E
:10745C003D30780068656C6C6F20776F726C640DD2
:10746C0000000000534F535F4B455920E69DBEE58D
:10747C00BC800D00534F535F4B455920E68C89E47B
:10748C00B88B0D004A5547455F4B455920E69DBECC
:10749C00E5BC800D000000004A5547455F4B45593F
:1074AC0020E68C89E4B88B0D000000000000000081
:1074BC000000000001020304060708090000000098
:1074CC000102030402030405060708090A0B0C0D4C
:1074DC000E0F101001020000020304050607080934
:1074EC000A0B0C0D0E0F101001025245454E542084
:1074FC006D616C6C6F632073756363656564656443
:10750C00002F6275696C642F676E752D746F6F6CCC
:10751C00732D666F722D73746D33325F31332E336E
:10752C002E72656C312E32303234303932362D3188
:10753C003731352F7372632F6E65776C69622F6EDE
:10754C0065776C69622F6C6962632F7374646C6904
:10755C00622F72616E642E63002C2066756E6374EC
:10756C00696F6E3A2000617373657274696F6E2077
:10757C0022257322206661696C65643A2066696C09
:10758C006520222573222C206C696E6520256425CC
:10759C007325730A00232D302B2000686C4C00657A
:1075AC006667454647003031323334353637383923
:1075BC004142434445460030313233343536373856
:1075CC003961626364656600002020202020202041
:1075DC002020282828282820202020202020202077
:1075EC002020202020202020208810101010101087
:1075FC0010101010101010101004040404040404D3
:10760C00040404101010101010104141414141416C
:10761C00010101010101010101010101010101014E
:10762C00010101011010101010104242424242425E
:10763C00020202020202020202020202020202021E
:10764C0002020202101010102000000000000000C6
:10765C00000000000000000000000000000000001E
:10766C00000000000000000000000000000000000E
:10767C0000000000000000000000000000000000FE
:10768C0000000000000000000000000000000000EE
:10769C0000000000000000000000000000000000DE
:1076AC0000000000000000000000000000000000CE
:1076BC0000000000000000000000000000000000BE
:0C76CC00000000000000000000000000B2
:0876D800748AFF7F010000002D
:0476E000310100086C
:0476E4000D0100088C
:1076E80000127A00100000000100000000000000F5
:1076F8009C720008AC720008BC7200080000000010
:1077080003000000C40500202C0000200000000039
:10771800C40500202C06002094060020000000006C
:107728000000000000000000000000000000000051
:107738000000000000000000000000000000000041
:107748000000000000000000000000000000000031
:08775800000000000000000029
:0400000508005A99FC
:00000001FF
